Stack Allocation = 16384 bytes

 SpDnd16

 Start     Length     Name                   Class
 0001:0000 0336AH     SEG_CODE_TEXT          CODE
 0001:336A 00000H     INSOBJ_TEXT            CODE
 0001:336A 00000H     ENUMFETC_TEXT          CODE
 0001:336A 00000H     OLE2UI_TEXT            CODE
 0001:336A 00000H     OLESTD_TEXT            CODE
 0001:336A 00000H     OLEUTL_TEXT            CODE
 0001:336A 00000H     COMMON_TEXT            CODE
 0001:336A 00000H     DRAWICON_TEXT          CODE
 0001:336A 00000H     ICON_TEXT              CODE
 0001:336A 00000H     ICONBOX_TEXT           CODE
 0001:336A 00000H     TARGTDEV_TEXT          CODE
 0001:336A 00000H     REGDB_TEXT             CODE
 0001:336A 00000H     RESIMAGE_TEXT          CODE
 0001:336A 00000H     UTILITY_TEXT           CODE
 0001:336A 00000H     GETICON_TEXT           CODE
 0001:336A 01FC1H     _TEXT                  CODE
 0001:5330 077F6H     COMDAT_SEG1            CODE
 0002:0000 00044H     SEG_CODE5_DATA         FAR_DATA
 0003:0000 00010H     NULL                   BEGDATA
 0003:0010 00B1EH     _DATA                  DATA
 0003:0B2E 00000H     XIFCB                  DATA
 0003:0B2E 00004H     XIFU                   DATA
 0003:0B32 00000H     XIFL                   DATA
 0003:0B32 00000H     XIFM                   DATA
 0003:0B32 00000H     XIFCE                  DATA
 0003:0B32 0000EH     CDATA                  DATA
 0003:0B40 00000H     XIFB                   DATA
 0003:0B40 00000H     XIF                    DATA
 0003:0B40 00000H     XIFE                   DATA
 0003:0B40 00000H     XIB                    DATA
 0003:0B40 00000H     XI                     DATA
 0003:0B40 00000H     XIE                    DATA
 0003:0B40 00000H     XPB                    DATA
 0003:0B40 00004H     XP                     DATA
 0003:0B44 00000H     XPE                    DATA
 0003:0B44 00000H     XCB                    DATA
 0003:0B44 00000H     XC                     DATA
 0003:0B44 00000H     XCE                    DATA
 0003:0B44 00000H     XCFB                   DATA
 0003:0B44 00000H     XCFCRT                 DATA
 0003:0B44 00000H     XCF                    DATA
 0003:0B44 00000H     XCFE                   DATA
 0003:0B44 00000H     DBDATA                 DATA
 0003:0B44 000E4H     IOB                    DATA
 0003:0C28 00000H     IOBX                   DATA
 0003:0C28 0000CH     IOBE                   DATA
 0003:0C34 000E4H     IOB2                   DATA
 0003:0D18 00000H     IOB2X                  DATA
 0003:0D18 0000CH     IOB2E                  DATA
 0003:0D24 00002H     CONST                  CONST
 0003:0D26 00008H     HDR                    MSG
 0003:0D2E 0018BH     MSG                    MSG
 0003:0EB9 00015H     PAD                    MSG
 0003:0ECE 00001H     EPAD                   MSG
 0003:0ED0 00B7AH     _BSS                   BSS
 0003:1A4A 00000H     XOB                    BSS
 0003:1A4A 00000H     XO                     BSS
 0003:1A4A 00000H     XOE                    BSS
 0003:1A4A 00000H     XOFB                   BSS
 0003:1A4A 00000H     XOF                    BSS
 0003:1A4A 00000H     XOFE                   BSS
 0003:1A50 00010H     c_common               BSS

 Origin   Group
 0003:0   DGROUP

 Address   Export                  Alias

 0001:4B0E ___ExportedStub         ___ExportedStub

  Address         Publics by Name

 0001:0F54       ??0CDataXferObj@@BEC@XZ
 0001:53AE       ??0CDropTarget@@REC@PEVCSimpleDoc@@@Z
 0001:0000       ??0CSimpleApp@@REC@XZ
 0001:0672       ??0CSimpleDoc@@REC@PEVCSimpleApp@@I@Z
 0001:29BE       ??0CSimpleSite@@REC@PEVCSimpleDoc@@@Z
 0001:0FC2       ??1CDataXferObj@@BEC@XZ
 0001:0052       ??1CSimpleApp@@REC@XZ
 0001:07A0       ??1CSimpleDoc@@REC@XZ
 0001:2AB8       ??1CSimpleSite@@REC@XZ
 0001:3454       ??2@ZAPEXI@Z
 0001:3442       ??3@ZAXPEX@Z
 0001:563A       ??_7CAdviseSink@@6F@
 0001:5506       ??_7CDataXferObj@@6F@
 0001:54D6       ??_7CDropSource@@6F@
 0001:54EA       ??_7CDropTarget@@6F@
 0001:55D2       ??_7COleClientSite@@6F@
 0001:533C       ??_7CSimpleApp@@6F@
 0001:54B6       ??_7CSimpleDoc@@6F@
 0001:565A       ??_7CSimpleSite@@6F@
 0001:55F6       ??_7IAdviseSink@@6F@
 0001:5536       ??_7IDataObject@@6F@
 0001:54C2       ??_7IDropSource@@6F@
 0001:549A       ??_7IDropTarget@@6F@
 0001:5616       ??_7IOleClientSite@@6F@
 0001:5330       ??_7IUnknown@@6F@
 0001:87F0       ??_C@_00A@?$AA@
 0001:75EC       ??_C@_01PCFE@?2?$AA@
 0001:768C       ??_C@_01POCP@?7?$AA@
 0001:C686       ??_C@_03DDP@CON?$AA@
 0001:C68A       ??_C@_03DLI@AUX?$AA@
 0001:C68E       ??_C@_03EHJD@PRN?$AA@
 0001:87F2       ??_C@_03NAME@?4?4?4?$AA@
 0001:9D6A       ??_C@_04CLJC@Font?$AA@
 0001:8800       ??_C@_04FOAE@?$CFd?$CF?$CF?$AA@
 0001:C674       ??_C@_04GNEC@COM2?$AA@
 0001:C662       ??_C@_04HLIF@LPT2?$AA@
 0001:C65C       ??_C@_04IEDM@LPT1?$AA@
 0001:C680       ??_C@_04JCDA@COM4?$AA@
 0001:C66E       ??_C@_04JCPL@COM1?$AA@
 0001:C67A       ??_C@_04MHNF@COM3?$AA@
 0001:96F4       ??_C@_04MOFI@?$CFs?$CFd?$AA@
 0001:C668       ??_C@_04NBBC@LPT3?$AA@
 0001:96B0       ??_C@_05FGFK@CLSID?$AA@
 0001:55CC       ??_C@_05NDCL@ias?4h?$AA@
 0001:5466       ??_C@_05NNFA@idt?4h?$AA@
 0001:7668       ??_C@_06HFAC@CLSID?2?$AA@
 0001:7660       ??_C@_06JPNA@?2CLSID?$AA@
 0001:972C       ??_C@_06KAHL@?$EA?$CFs?$CB?$CFs?$AA@
 0001:5596       ??_C@_06LNPM@iocs?4h?$AA@
 0001:96C0       ??_C@_07CPIP@Package?$AA@
 0001:B75A       ??_C@_07LGIJ@DISPLAY?$AA@
 0001:BAE6       ??_C@_08BJKM@CLSID?2?$CFs?$AA@
 0001:87A8       ??_C@_08NJLM@FileName?$AA@
 0001:87F6       ??_C@_09DKHB@Structure?$AA@
 0001:96B6       ??_C@_09JJAI@Linked?5?$CFs?$AA@
 0001:9952       ??_C@_09LHIP@Embedding?$AA@
 0001:879E       ??_C@_09NJ@OwnerLink?$AA@
 0001:8782       ??_C@_0BA@IEJA@Embedded?5Object?$AA@
 0001:C61E       ??_C@_0BA@JEHM@GetOpenFileName?$AA@
 0001:BAF0       ??_C@_0BA@LJEI@?2AuxUserType?2?$CFd?$AA@
 0001:86F4       ??_C@_0BB@PGGH@OLEUI_MSG_BROWSE?$AA@
 0001:874A       ??_C@_0BC@GMEI@Object?5Descriptor?$AA@
 0001:871C       ??_C@_0BD@HNAP@commdlg_FileNameOK?$AA@
 0001:86E0       ??_C@_0BE@FEHN@OLEUI_MSG_ENDDIALOG?$AA@
 0001:CAE6       ??_C@_0BE@GGIG@?2Shell?2Open?2Command?$AA@
 0001:8706       ??_C@_0BF@COIE@OLEUI_MSG_CHANGEICON?$AA@
 0001:C62E       ??_C@_0BF@GCFH@CommDlgExtendedError?$AA@
 0001:55B6       ??_C@_0BG@BCJB@In?5IAS?8s?5destructor?$AN?6?$AA@
 0001:5484       ??_C@_0BG@DGDH@In?5IDS?8s?5destructor?$AN?6?$AA@
 0001:5450       ??_C@_0BG@NDHK@In?5IDT?8s?5destructor?$AN?6?$AA@
 0001:5438       ??_C@_0BH@FLKL@In?5IDT?8s?5constructor?$AN?6?$AA@
 0001:875C       ??_C@_0BH@FOOO@Link?5Source?5Descriptor?$AA@
 0001:546C       ??_C@_0BH@JHEO@In?5IDS?8s?5constructor?$AN?6?$AA@
 0001:559E       ??_C@_0BH@NFGK@In?5IAS?8s?5constructor?$AN?6?$AA@
 0001:557E       ??_C@_0BH@PEFE@In?5IOCS?8s?5destructor?$AN?6?$AA@
 0001:5566       ??_C@_0BI@IJIM@In?5IOCS?8s?5constructor?$AN?6?$AA@
 0001:8730       ??_C@_0BK@LOCD@OLEUI_MSG_CLOSEBUSYDIALOG?$AA@
 0001:CAFA       ??_C@_0BP@CLAL@Protocol?2StdFileEditing?2Server?$AA@
 0001:7634       ??_C@_0CA@PANP@?2protocol?2StdFileEditing?2server?$AA@
 0001:BB0C       ??_C@_0CB@FCAE@CLSID?2?$CFs?2DataFormats?2DefaultFile@
 0001:87CA       ??_C@_0CG@HCKA@resource?5read?50x?$CFX?0?5my?5value?5is?5@
 0001:75EE       ??_C@_0CH@JMMM@?$CK?$CK?$CK?5Please?5install?5VC?$CL?$CL?5Patch?5?$CD1@
 0001:96C8       ??_C@_0CL@HONB@ERROR?3?5INTERFACE?5METHOD?5NOT?5IMPL@
 0001:96FA       ??_C@_0DC@GEMK@OleStdCreateTempFileMoniker?3?5Mon@
 0001:9676       ??_C@_0DJ@NHNH@OleStdSwitchDisplayAspect?3?5Cache@
 0001:B324       ??_C@_0L@CPGB@HWND_CIDLG?$AA@
 0001:C650       ??_C@_0L@KCEB@?$CFc?$CFc?$CFc?4?4?4?2?$AA@
 0001:BB00       ??_C@_0M@BODG@?2MiscStatus?$AA@
 0001:87BE       ??_C@_0M@GHPL@ole2uiIBCls?$AA@
 0001:C644       ??_C@_0M@JEJD@LocalServer?$AA@
 0001:CB1A       ??_C@_0M@JONA@DefaultIcon?$AA@
 0001:8792       ??_C@_0M@KPGD@Link?5Source?$AA@
 0001:75D2       ??_C@_0M@LNGB@COMMDLG?4DLL?$AA@
 0001:87B2       ??_C@_0M@MBIN@ole2uiRICls?$AA@
 0001:7654       ??_C@_0M@PKFG@?2Insertable?$AA@
 0001:7616       ??_C@_0N@IIFK@commdlg_help?$AA@
 0001:8774       ??_C@_0N@LHIH@Embed?5Source?$AA@
 0001:86C2       ??_C@_0N@OCMF@VERIFICATION?$AA@
 0001:7670       ??_C@_0N@OIGG@?2LocalServer?$AA@
 0001:75DE       ??_C@_0N@PNI@GetFileTitle?$AA@
 0001:542A       ??_C@_0O@GKMD@m_nCount?5?$DN?$DN?50?$AA@
 0001:767E       ??_C@_0O@JEDJ@?2InProcServer?$AA@
 0001:86D0       ??_C@_0P@LMIA@OLEUI_MSG_HELP?$AA@
 0001:7624       ??_C@_0P@PDBJ@?2NotInsertable?$AA@
 0001:267A       ?About@@ZCHIIGJ@Z
 0001:1520       ?AddRef@CAdviseSink@@VEAKXZ
 0001:10B6       ?AddRef@CDataXferObj@@VEAKXZ
 0001:17CE       ?AddRef@CDropSource@@VEAKXZ
 0001:1EBA       ?AddRef@CDropTarget@@VEAKXZ
 0001:2202       ?AddRef@COleClientSite@@VEAKXZ
 0001:00C4       ?AddRef@CSimpleApp@@VEAKXZ
 0001:09AC       ?AddRef@CSimpleDoc@@VEAKXZ
 0001:2D4E       ?AddRef@CSimpleSite@@VEAKXZ
 0001:0602       ?Close@CSimpleDoc@@RECXXZ
 0001:2B98       ?CloseOleObject@CSimpleSite@@RECXXZ
 0001:0C60       ?CopyObjectToClip@CSimpleDoc@@RECXXZ
 0001:0D68       ?Create@CDataXferObj@@TAPEV1@PEVCSimpleSite@@PEUtagPOINTL@@@Z
 0001:04D6       ?Create@CSimpleDoc@@TAPEV1@PEVCSimpleApp@@PEUtagRECT@@I@Z
 0001:28FE       ?Create@CSimpleSite@@TAPEV1@PEVCSimpleDoc@@@Z
 0001:5348       ?DAdvise@CDataXferObj@@VEAPEXPEUtagFORMATETC@@KPEUIAdviseSink@@PEK@Z
 0001:0082       ?DestroyDocs@CSimpleApp@@RECXXZ
 0001:0C12       ?DisableInsertObject@CSimpleDoc@@RECXXZ
 0001:26B2       ?DocWndProc@@ZCJIIIJ@Z
 0001:16C8       ?DoDragDrop@CSimpleDoc@@RECKXZ
 0001:19B6       ?DoDragScroll@CDropTarget@@BECHUtagPOINTL@@@Z
 0001:1F22       ?DragEnter@CDropTarget@@VEAPEXPEUIDataObject@@KUtagPOINTL@@PEK@Z
 0001:2050       ?DragLeave@CDropTarget@@VEAPEXXZ
 0001:1FD6       ?DragOver@CDropTarget@@VEAPEXKUtagPOINTL@@PEK@Z
 0001:1DB8       ?DrawDragFeedback@CDropTarget@@BECXUtagPOINTL@@@Z
 0001:2074       ?Drop@CDropTarget@@VEAPEXPEUIDataObject@@KUtagPOINTL@@PEK@Z
 0001:535A       ?DUnadvise@CDataXferObj@@VEAPEXK@Z
 0001:536C       ?EnumDAdvise@CDataXferObj@@VEAPEXPEPEUIEnumSTATDATA@@@Z
 0001:11C8       ?EnumFormatEtc@CDataXferObj@@VEAPEXKPEPEUIEnumFORMATETC@@@Z
 0003:06CC       ?fBeVerbose@@3HE
 0001:0134       ?fInitApplication@CSimpleApp@@RECHI@Z
 0001:01F0       ?fInitInstance@CSimpleApp@@RECHIH@Z
 0001:537E       ?GetCanonicalFormatEtc@CDataXferObj@@VEAPEXPEUtagFORMATETC@@0@Z
 0001:233A       ?GetContainer@COleClientSite@@VEAPEXPEPEUIOleContainer@@@Z
 0001:123C       ?GetData@CDataXferObj@@VEAPEXPEUtagFORMATETC@@PEUtagSTGMEDIUM@@@Z
 0001:1402       ?GetDataHere@CDataXferObj@@VEAPEXPEUtagFORMATETC@@PEUtagSTGMEDIUM@@@Z
 0001:2310       ?GetMoniker@COleClientSite@@VEAPEXKKPEPEUIMoniker@@@Z
 0001:30BA       ?GetObjRect@CSimpleSite@@RECXPEUtagRECT@@@Z
 0001:185E       ?GiveFeedback@CDropSource@@VEAPEXK@Z
 0003:0ED0       ?g_cfEmbeddedObject@@3GE
 0003:0ED2       ?g_cfObjectDescriptor@@3GE
 0001:04AC       ?HandleAccelerators@CSimpleApp@@RECHPEUtagMSG@@@Z
 0001:1C3C       ?InitDragFeedback@CDropTarget@@BECXPEUIDataObject@@UtagPOINTL@@@Z
 0001:2DBE       ?InitObject@CSimpleSite@@RECPEXH@Z
 0001:0A1C       ?InsertObject@CSimpleDoc@@RECXXZ
 0001:0B86       ?lAddVerbs@CSimpleDoc@@RECJXZ
 0001:02FE       ?lCommandHandler@CSimpleApp@@RECJIIIJ@Z
 0001:0476       ?lCreateDoc@CSimpleApp@@RECJIIIJ@Z
 0003:0ED4       ?lpCSimpleApp@@3PEVCSimpleApp@@E
 0001:0B5C       ?lResizeDoc@CSimpleDoc@@RECJPEUtagRECT@@@Z
 0001:0448       ?lSizeHandler@CSimpleApp@@RECJIIIJ@Z
 0001:2566       ?MainWndProc@@ZCJIIIJ@Z
 0001:166E       ?OnClose@CAdviseSink@@VEAXXZ
 0001:1588       ?OnDataChange@CAdviseSink@@VEAXPEUtagFORMATETC@@PEUtagSTGMEDIUM@@@Z
 0001:163E       ?OnRename@CAdviseSink@@VEAXPEUIMoniker@@@Z
 0001:1656       ?OnSave@CAdviseSink@@VEAXXZ
 0001:237E       ?OnShowWindow@COleClientSite@@VEAPEXH@Z
 0001:15A0       ?OnViewChange@CAdviseSink@@VEAXKJ@Z
 0001:04B2       ?PaintApp@CSimpleApp@@RECXI@Z
 0001:0BEE       ?PaintDoc@CSimpleDoc@@RECXI@Z
 0001:2F4E       ?PaintObj@CSimpleSite@@RECXI@Z
 0001:1836       ?QueryContinueDrag@CDropSource@@VEAPEXHK@Z
 0001:1686       ?QueryDrag@CSimpleDoc@@RECHUtagPOINT@@@Z
 0001:1870       ?QueryDrop@CDropTarget@@BECHKUtagPOINTL@@HPEK@Z
 0001:1126       ?QueryGetData@CDataXferObj@@VEAPEXPEUtagFORMATETC@@@Z
 0001:14E4       ?QueryInterface@CAdviseSink@@VEAPEXAFUGUID@@PEPEX@Z
 0001:1032       ?QueryInterface@CDataXferObj@@VEAPEXAFUGUID@@PEPEX@Z
 0001:1792       ?QueryInterface@CDropSource@@VEAPEXAFUGUID@@PEPEX@Z
 0001:1E7E       ?QueryInterface@CDropTarget@@VEAPEXAFUGUID@@PEPEX@Z
 0001:21C6       ?QueryInterface@COleClientSite@@VEAPEXAFUGUID@@PEPEX@Z
 0001:009A       ?QueryInterface@CSimpleApp@@VEAPEXAFUGUID@@PEPEX@Z
 0001:08D8       ?QueryInterface@CSimpleDoc@@VEAPEXAFUGUID@@PEPEX@Z
 0001:2C7A       ?QueryInterface@CSimpleSite@@VEAPEXAFUGUID@@PEPEX@Z
 0001:1554       ?Release@CAdviseSink@@VEAKXZ
 0001:10DA       ?Release@CDataXferObj@@VEAKXZ
 0001:1802       ?Release@CDropSource@@VEAKXZ
 0001:1EEE       ?Release@CDropTarget@@VEAKXZ
 0001:2236       ?Release@COleClientSite@@VEAKXZ
 0001:00E8       ?Release@CSimpleApp@@VEAKXZ
 0001:09D0       ?Release@CSimpleDoc@@VEAKXZ
 0001:2D72       ?Release@CSimpleSite@@VEAKXZ
 0001:23EE       ?RequestNewObjectLayout@COleClientSite@@VEAPEXXZ
 0001:226A       ?SaveObject@COleClientSite@@VEAPEXXZ
 0001:539C       ?SetData@CDataXferObj@@VEAPEXPEUtagFORMATETC@@PEUtagSTGMEDIUM@@H@Z
 0001:2364       ?ShowObject@COleClientSite@@VEAPEXXZ
 0001:30F6       ?StartTest1@@ZAXPEVCSimpleApp@@@Z
 0001:3208       ?StartTest2@@ZAXPEVCSimpleApp@@@Z
 0001:1D5C       ?UndrawDragFeedback@CDropTarget@@BECXXZ
 0001:2BD0       ?UnloadOleObject@CSimpleSite@@RECXXZ
 0000:0000  Imp  ANSINEXT             (USER.472)
 0000:0000  Imp  ANSIPREV             (USER.473)
 0000:0000  Imp  ANSITOOEM            (KEYBOARD.5)
 0000:0000  Imp  BEGINPAINT           (USER.39)
 0000:0000  Imp  BITBLT               (GDI.34)
 0000:0000  Imp  BRINGWINDOWTOTOP     (USER.45)
 0001:BF60       BROWSE
 0001:A5BA       CHANGEICONDIALOGPROC
 0000:0000  Imp  CHECKDLGBUTTON       (USER.97)
 0000:0000  Imp  CHECKRADIOBUTTON     (USER.96)
 0000:0000  Unr  CHOPTEXT
 0000:0000  Imp  CLOSEMETAFILE        (GDI.126)
 0000:0000  Imp  CLSIDFROMPROGID      (COMPOBJ.61)
 0000:0000  Imp  CLSIDFROMSTRING      (COMPOBJ.20)
 0000:0000  Imp  CODOSDATETIMETOFILETIME (COMPOBJ.31)
 0000:0000  Imp  COFILETIMENOW        (COMPOBJ.82)
 0000:0000  Imp  COGETMALLOC          (COMPOBJ.4)
 0000:0000  Imp  COISOLE1CLASS        (COMPOBJ.36)
 0000:0000  Imp  COLOCKOBJECTEXTERNAL (COMPOBJ.63)
 0000:0000  Imp  COTREATASCLASS       (COMPOBJ.66)
 0000:0000  Imp  CREATEBINDCTX        (OLE2.26)
 0000:0000  Imp  CREATEBITMAP         (GDI.48)
 0000:0000  Imp  CREATECOMPATIBLEBITMAP (GDI.51)
 0000:0000  Imp  CREATECOMPATIBLEDC   (GDI.52)
 0000:0000  Imp  CREATEDC             (GDI.53)
 0000:0000  Imp  CREATEFILEMONIKER    (OLE2.28)
 0000:0000  Imp  CREATEFONTINDIRECT   (GDI.57)
 0000:0000  Imp  CREATEHATCHBRUSH     (GDI.58)
 0000:0000  Imp  CREATEIC             (GDI.153)
 0000:0000  Imp  CREATEICON           (USER.407)
 0000:0000  Imp  CREATEILOCKBYTESONHGLOBAL (OLE2.54)
 0000:0000  Imp  CREATEMETAFILE       (GDI.125)
 0000:0000  Imp  CREATEPALETTE        (GDI.360)
 0000:0000  Imp  CREATEPEN            (GDI.61)
 0000:0000  Imp  CREATEPOPUPMENU      (USER.415)
 0000:0000  Imp  CREATESOLIDBRUSH     (GDI.66)
 0000:0000  Imp  CREATESTREAMONHGLOBAL (OLE2.84)
 0000:0000  Imp  CREATEWINDOW         (USER.41)
 0000:0000  Imp  DEFWINDOWPROC        (USER.107)
 0000:0000  Imp  DELETEDC             (GDI.68)
 0000:0000  Imp  DELETEMENU           (USER.413)
 0000:0000  Imp  DELETEMETAFILE       (GDI.127)
 0000:0000  Imp  DELETEOBJECT         (GDI.69)
 0000:0000  Imp  DESTROYICON          (USER.457)
 0000:0000  Imp  DESTROYMENU          (USER.152)
 0000:0000  Imp  DESTROYWINDOW        (USER.53)
 0000:0000  Imp  DIALOGBOX            (USER.87)
 0000:0000  Imp  DIALOGBOXINDIRECTPARAM (USER.240)
 0000:0000  Imp  DIALOGBOXPARAM       (USER.239)
 0000:0000  Imp  DISPATCHMESSAGE      (USER.114)
 0000:0000  Imp  DODRAGDROP           (OLE2.37)
 0001:C5AE       DOESFILEEXIST
 0000:0000  Imp  DOS3CALL             (KERNEL.102)
 0000:0000  Imp  DRAWFOCUSRECT        (USER.466)
 0000:0000  Imp  DRAWICON             (USER.84)
 0000:0000  Imp  ENABLEMENUITEM       (USER.155)
 0000:0000  Imp  ENABLEWINDOW         (USER.34)
 0000:0000  Imp  ENDDIALOG            (USER.88)
 0000:0000  Imp  ENDPAINT             (USER.40)
 0000:0000  Imp  ENUMMETAFILE         (GDI.175)
 0001:A142       ENUMMETAFILEEXTRACTICON
 0001:A412       ENUMMETAFILEEXTRACTICONSOURCE
 0001:A000       ENUMMETAFILEEXTRACTLABEL
 0001:9ECC       ENUMMETAFILEICONDRAW
 0001:C104       ERRORWITHFILE
 0000:0000  Imp  EXTRACTICON          (SHELL.34)
 0000:0000  Imp  EXTTEXTOUT           (GDI.351)
 0000:0000  Imp  FATALAPPEXIT         (KERNEL.137)
 0000:0000  Imp  FATALEXIT            (KERNEL.1)
 0001:C7D4       FICONFILEFROMCLASS
 0000:0000  Imp  FILLRECT             (USER.81)
 0000:0000  Imp  FINDRESOURCE         (KERNEL.60)
 0000:0000  Imp  FREELIBRARY          (KERNEL.96)
 0000:0000  Imp  FREEPROCINSTANCE     (KERNEL.52)
 0000:0000  Imp  FREERESOURCE         (KERNEL.63)
 0000:0000  Unr  FSERVERFROMCLASS
 0001:C692       GETASSOCIATEDEXECUTABLE
 0000:0000  Imp  GETBITMAPBITS        (GDI.74)
 0000:0000  Imp  GETBKCOLOR           (GDI.75)
 0000:0000  Imp  GETCLASSFILE         (OLE2.57)
 0000:0000  Imp  GETCLIENTRECT        (USER.33)
 0000:0000  Imp  GETCURRENTTIME       (USER.15)
 0000:0000  Imp  GETDC                (USER.66)
 0000:0000  Imp  GETDEVICECAPS        (GDI.80)
 0000:0000  Imp  GETDIALOGBASEUNITS   (USER.243)
 0000:0000  Imp  GETDLGITEM           (USER.91)
 0000:0000  Imp  GETDLGITEMTEXT       (USER.93)
 0000:0000  Imp  GETDOSENVIRONMENT    (KERNEL.131)
 0000:0000  Imp  GETFOCUS             (USER.23)
 0000:0000  Imp  GETMENU              (USER.157)
 0000:0000  Imp  GETMENUITEMCOUNT     (USER.263)
 0000:0000  Imp  GETMESSAGE           (USER.108)
 0000:0000  Imp  GETMODULEFILENAME    (KERNEL.49)
 0000:0000  Imp  GETOBJECT            (GDI.82)
 0000:0000  Imp  GETPARENT            (USER.46)
 0000:0000  Imp  GETPROCADDRESS       (KERNEL.50)
 0000:0000  Imp  GETPROFILEINT        (KERNEL.57)
 0000:0000  Imp  GETPROP              (USER.25)
 0000:0000  Imp  GETRUNNINGOBJECTTABLE (OLE2.30)
 0000:0000  Imp  GETSTOCKOBJECT       (GDI.87)
 0000:0000  Imp  GETSUBMENU           (USER.159)
 0000:0000  Imp  GETSYSCOLOR          (USER.180)
 0000:0000  Imp  GETSYSTEMMETRICS     (USER.179)
 0000:0000  Imp  GETTEXTEXTENTPOINT   (GDI.471)
 0000:0000  Imp  GETVERSION           (KERNEL.3)
 0000:0000  Imp  GETWINDOWRECT        (USER.32)
 0000:0000  Imp  GETWINDOWTEXT        (USER.36)
 0000:0000  Imp  GETWINDOWWORD        (USER.133)
 0000:0000  Imp  GLOBALALLOC          (KERNEL.15)
 0000:0000  Imp  GLOBALFREE           (KERNEL.17)
 0000:0000  Imp  GLOBALLOCK           (KERNEL.18)
 0000:0000  Imp  GLOBALREALLOC        (KERNEL.16)
 0000:0000  Imp  GLOBALSIZE           (KERNEL.20)
 0000:0000  Imp  GLOBALUNLOCK         (KERNEL.19)
 0000:0000  Unr  HICONANDSOURCEFROMCLASS
 0000:0000  Unr  HICONFROMCLASS
 0001:BF4A       HOURGLASSOFF
 0001:BF2A       HOURGLASSON
 0001:B3A8       ICONBOXWNDPROC
 0000:0000  Imp  INFLATERECT          (USER.78)
 0000:0000  Imp  INITAPP              (USER.5)
 0000:0000  Imp  INITTASK             (KERNEL.91)
 0000:0000  Imp  INSERTMENU           (USER.410)
 0001:598C       INSERTOBJECTDIALOGPROC
 0000:0000  Imp  INVALIDATERECT       (USER.125)
 0000:0000  Imp  ISBADCODEPTR         (KERNEL.336)
 0000:0000  Imp  ISBADREADPTR         (KERNEL.334)
 0000:0000  Imp  ISBADWRITEPTR        (KERNEL.335)
 0000:0000  Imp  ISDBCSLEADBYTE       (KERNEL.207)
 0000:0000  Imp  ISDIALOGMESSAGE      (USER.90)
 0000:0000  Imp  ISDLGBUTTONCHECKED   (USER.98)
 0000:0000  Imp  ISEQUALGUID          (COMPOBJ.18)
 0000:0000  Imp  ISWINDOW             (USER.47)
 0000:0000  Imp  KILLTIMER            (USER.12)
 0000:0000  Imp  LOADBITMAP           (USER.175)
 0000:0000  Imp  LOADCURSOR           (USER.173)
 0000:0000  Imp  LOADICON             (USER.174)
 0000:0000  Imp  LOADLIBRARY          (KERNEL.95)
 0000:0000  Imp  LOADRESOURCE         (KERNEL.61)
 0000:0000  Imp  LOADSTRING           (USER.176)
 0000:0000  Imp  LOCKRESOURCE         (KERNEL.62)
 0000:0000  Imp  LOCKSEGMENT          (KERNEL.23)
 0001:9C08       LPVSTANDARDENTRY
 0001:9B4A       LPVSTANDARDINIT
 0000:0000  Imp  LSTRCAT              (KERNEL.89)
 0000:0000  Imp  LSTRCMP              (USER.430)
 0000:0000  Imp  LSTRCMPI             (USER.471)
 0000:0000  Imp  LSTRCPY              (KERNEL.88)
 0000:0000  Imp  LSTRCPYN             (KERNEL.353)
 0000:0000  Imp  LSTRLEN              (KERNEL.90)
 0000:0000  Imp  MAKEPROCINSTANCE     (KERNEL.51)
 0000:0000  Imp  MESSAGEBOX           (USER.1)
 0000:0000  Imp  MKPARSEDISPLAYNAME   (OLE2.23)
 0000:0000  Imp  MOVEWINDOW           (USER.56)
 0000:0000  Imp  MULDIV               (GDI.128)
 0000:0000  Imp  OEMTOANSI            (KEYBOARD.6)
 0000:0000  Imp  OFFSETRECT           (USER.77)
 0000:0000  Imp  OLEBUILDVERSION      (OLE2.1)
 0000:0000  Imp  OLECREATE            (OLE2.10)
 0000:0000  Imp  OLECREATEFROMDATA    (OLE2.8)
 0000:0000  Imp  OLECREATEFROMFILE    (OLE2.67)
 0000:0000  Imp  OLECREATELINKTOFILE  (OLE2.68)
 0000:0000  Imp  OLEDRAW              (OLE2.58)
 0000:0000  Imp  OLEDUPLICATEDATA     (OLE2.51)
 0000:0000  Imp  OLEFLUSHCLIPBOARD    (OLE2.76)
 0000:0000  Imp  OLEGETICONOFCLASS    (OLE2.53)
 0000:0000  Imp  OLEGETICONOFFILE     (OLE2.52)
 0000:0000  Imp  OLEINITIALIZE        (OLE2.2)
 0000:0000  Imp  OLELOAD              (OLE2.12)
 0000:0000  Imp  OLEMETAFILEPICTFROMICONANDLABEL (OLE2.56)
 0000:0000  Imp  OLEQUERYCREATEFROMDATA (OLE2.7)
 0000:0000  Imp  OLEQUERYLINKFROMDATA (OLE2.6)
 0000:0000  Imp  OLESAVE              (OLE2.13)
 0000:0000  Imp  OLESAVETOSTREAM      (OLE2.24)
 0000:0000  Imp  OLESETCLIPBOARD      (OLE2.49)
 0000:0000  Imp  OLESETCONTAINEDOBJECT (OLE2.86)
 0000:0000  Unr  OLESTDCHECKVTBL
 0000:0000  Unr  OLESTDCOMMITSTORAGE
 0001:B622       OLESTDCOMPAREFORMATETC
 0001:B6F0       OLESTDCOMPARETARGETDEVICE
 0001:B584       OLESTDCOPYFORMATETC
 0001:8A4A       OLESTDCOPYSTRING
 0001:B532       OLESTDCOPYTARGETDEVICE
 0000:0000  Unr  OLESTDCREATECHILDSTORAGE
 0000:0000  Unr  OLESTDCREATEDC
 0000:0000  Unr  OLESTDCREATEIC
 0000:0000  Unr  OLESTDCREATEROOTSTORAGE
 0001:8AD4       OLESTDCREATESTORAGEONHGLOBAL
 0000:0000  Unr  OLESTDCREATETARGETDEVICE
 0000:0000  Unr  OLESTDCREATETEMPFILEMONIKER
 0001:8B6C       OLESTDCREATETEMPSTORAGE
 0000:0000  Unr  OLESTDDELETETARGETDEVICE
 0000:0000  Unr  OLESTDDESTROYALLELEMENTS
 0000:0000  Unr  OLESTDDOCONVERT
 0000:0000  Unr  OLESTDDOTREATASCLASS
 0001:768E       OLESTDENUMFMTETC_CREATE
 0000:0000  Unr  OLESTDFILLOBJECTDESCRIPTORFROMDATA
 0001:899E       OLESTDFREE
 0001:89F4       OLESTDFREESTRING
 0000:0000  Unr  OLESTDGETAUXUSERTYPE
 0001:8844       OLESTDGETDATA
 0001:BA08       OLESTDGETDEFAULTFILEFORMATOFCLASS
 0001:9416       OLESTDGETFIRSTMONIKER
 0000:0000  Unr  OLESTDGETITEMTOKEN
 0000:0000  Unr  OLESTDGETLENFILEPREFIXOFMONIKER
 0000:0000  Unr  OLESTDGETLINKSOURCEDATA
 0001:91D6       OLESTDGETMETAFILEPICTFROMOLEOBJECT
 0000:0000  Unr  OLESTDGETMISCSTATUSOFCLASS
 0001:8CD4       OLESTDGETOBJECTDESCRIPTORDATA
 0001:8E5A       OLESTDGETOBJECTDESCRIPTORDATAFROMOLEOBJECT
 0001:8BCA       OLESTDGETOLEOBJECTDATA
 0000:0000  Unr  OLESTDGETPRIORITYCLIPBOARDFORMAT
 0000:0000  Unr  OLESTDGETSIZE
 0000:0000  Unr  OLESTDGETTREATASFMTUSERTYPE
 0001:B884       OLESTDGETUSERTYPEOFCLASS
 0000:0000  Unr  OLESTDICONLABELTEXTOUT
 0000:0000  Unr  OLESTDINITVTBL
 0000:0000  Unr  OLESTDISDUPLICATEFORMAT
 0000:0000  Unr  OLESTDISOLELINK
 0001:8940       OLESTDMALLOC
 0001:94CC       OLESTDMARKPASTEENTRYLIST
 0000:0000  Unr  OLESTDMKPARSEDISPLAYNAME
 0000:0000  Unr  OLESTDNOTEFILECHANGETIME
 0000:0000  Unr  OLESTDNOTEOBJECTCHANGETIME
 0000:0000  Unr  OLESTDOPENCHILDSTORAGE
 0000:0000  Unr  OLESTDOPENORCREATEROOTSTORAGE
 0000:0000  Unr  OLESTDOPENROOTSTORAGE
 0001:8806       OLESTDQUERYINTERFACE
 0000:0000  Unr  OLESTDREALLOC
 0000:0000  Unr  OLESTDREGISTERASRUNNING
 0001:936E       OLESTDRELEASE
 0000:0000  Unr  OLESTDREVOKEASRUNNING
 0000:0000  Unr  OLESTDSETICONINCACHE
 0000:0000  Unr  OLESTDSETUPADVISES
 0000:0000  Unr  OLESTDSWITCHDISPLAYASPECT
 0001:934A       OLESTDVERIFYRELEASE
 0001:7CD4       OLEUIADDVERBMENU
 0000:0000  Unr  OLEUICANUNLOADNOW
 0001:A518       OLEUICHANGEICON
 0001:7B38       OLEUIINITIALIZE
 0001:5666       OLEUIINSERTOBJECT
 0001:A0DE       OLEUIMETAFILEPICTEXTRACTICON
 0001:A36E       OLEUIMETAFILEPICTEXTRACTICONSOURCE
 0001:9F48       OLEUIMETAFILEPICTEXTRACTLABEL
 0001:9DB8       OLEUIMETAFILEPICTICONDRAW
 0001:9D70       OLEUIMETAFILEPICTICONFREE
 0001:7CBC       OLEUIUNINITIALIZE
 0000:0000  Unr  OLEUIUPDATELINKS
 0000:0000  Imp  OLEUNINITIALIZE      (OLE2.3)
 0000:0000  Imp  OPENFILE             (KERNEL.74)
 0001:C200       OPENFILEERROR
 0000:0000  Imp  OUTPUTDEBUGSTRING    (KERNEL.115)
 0000:0000  Unr  PARSECMDLINE
 0000:0008  Abs  pAtomTable
 0000:0000  Imp  PEEKMESSAGE          (USER.109)
 0000:0000  Imp  PLAYMETAFILE         (GDI.123)
 0000:0000  Imp  PLAYMETAFILERECORD   (GDI.176)
 0000:0006  Abs  pLocalHeap
 0001:C796       POINTERTONTHFIELD
 0000:0000  Imp  POSTMESSAGE          (USER.110)
 0000:0000  Imp  POSTQUITMESSAGE      (USER.6)
 0000:0000  Imp  PROGIDFROMCLSID      (COMPOBJ.62)
 0001:829E       PROMPTUSERDLGPROC
 0000:000E  Abs  pStackBot
 0000:000C  Abs  pStackMin
 0000:000A  Abs  pStackTop
 0000:0000  Imp  PTINRECT             (USER.76)
 0000:0000  Imp  READCLASSSTG         (OLE2.18)
 0000:0000  Imp  READFMTUSERTYPESTG   (OLE2.74)
 0000:0000  Imp  REALIZEPALETTE       (USER.283)
 0000:0000  Imp  RECTANGLE            (GDI.27)
 0000:0000  Imp  REGCLOSEKEY          (SHELL.3)
 0000:0000  Imp  REGENUMKEY           (SHELL.7)
 0000:0000  Imp  REGISTERCLASS        (USER.57)
 0000:0000  Imp  REGISTERCLIPBOARDFORMAT (USER.145)
 0000:0000  Imp  REGISTERDRAGDROP     (OLE2.35)
 0000:0000  Imp  REGISTERWINDOWMESSAGE (USER.118)
 0000:0000  Imp  REGOPENKEY           (SHELL.1)
 0000:0000  Imp  REGQUERYVALUE        (SHELL.6)
 0000:0000  Imp  REGSETVALUE          (SHELL.5)
 0000:0000  Imp  RELEASECAPTURE       (USER.19)
 0000:0000  Imp  RELEASEDC            (USER.68)
 0000:0000  Imp  RELEASESTGMEDIUM     (OLE2.32)
 0000:0000  Imp  REMOVEMENU           (USER.412)
 0000:0000  Imp  REMOVEPROP           (USER.24)
 0001:C0CE       REPLACECHARWITHNULL
 0000:0000  Unr  RESETORIGDC
 0000:0000  Imp  RESTOREDC            (GDI.39)
 0001:BC30       RESULTIMAGEWNDPROC
 0000:0000  Imp  REVOKEDRAGDROP       (OLE2.36)
 0003:0004       rsrvptrs
 0000:0000  Imp  SAVEDC               (GDI.30)
 0000:0000  Imp  SCREENTOCLIENT       (USER.29)
 0000:0000  Imp  SELECTOBJECT         (GDI.45)
 0000:0000  Imp  SELECTPALETTE        (USER.282)
 0000:0000  Imp  SENDDLGITEMMESSAGE   (USER.101)
 0000:0000  Imp  SENDMESSAGE          (USER.111)
 0000:0000  Imp  SETBKCOLOR           (GDI.1)
 0000:0000  Imp  SETBRUSHORG          (GDI.148)
 0000:0000  Imp  SETCAPTURE           (USER.18)
 0000:0000  Imp  SETCONVERTSTG        (OLE2.83)
 0000:0000  Imp  SETCURSOR            (USER.69)
 0000:0000  Unr  SETDCTOANISOTROPIC
 0000:0000  Unr  SETDCTODRAWINHIMETRICRECT
 0000:0000  Imp  SETDIBITS            (GDI.440)
 0000:0000  Imp  SETDLGITEMTEXT       (USER.92)
 0000:0000  Imp  SETFOCUS             (USER.22)
 0000:0000  Imp  SETMAPMODE           (GDI.3)
 0000:0000  Imp  SETMESSAGEQUEUE      (USER.266)
 0000:0000  Imp  SETPROP              (USER.26)
 0000:0000  Imp  SETROP2              (GDI.4)
 0000:0000  Imp  SETTEXTCOLOR         (GDI.9)
 0000:0000  Imp  SETTIMER             (USER.10)
 0000:0000  Imp  SETVIEWPORTEXTEX     (GDI.479)
 0000:0000  Imp  SETVIEWPORTORGEX     (GDI.480)
 0000:0000  Imp  SETWINDOWEXTEX       (GDI.481)
 0000:0000  Imp  SETWINDOWORGEX       (GDI.482)
 0000:0000  Imp  SETWINDOWPOS         (USER.232)
 0000:0000  Imp  SETWINDOWTEXT        (USER.37)
 0000:0000  Imp  SETWINDOWWORD        (USER.134)
 0000:0000  Imp  SHOWCURSOR           (USER.71)
 0000:0000  Imp  SHOWWINDOW           (USER.42)
 0001:9CC4       STANDARDCLEANUP
 0001:9D14       STANDARDSHOWDLGITEM
 0000:0000  Imp  STGCREATEDOCFILE     (STORAGE.1)
 0000:0000  Imp  STGCREATEDOCFILEONILOCKBYTES (STORAGE.2)
 0000:0000  Imp  STGOPENSTORAGE       (STORAGE.3)
 0000:0000  Imp  STRINGFROMCLSID      (COMPOBJ.19)
 0000:0000  Imp  TRANSLATEMESSAGE     (USER.113)
 0000:0000  Unr  UCLASSFROMDESCRIPTION
 0000:0000  Unr  UDESCRIPTIONFROMCLASS
 0000:0000  Imp  UNREALIZEOBJECT      (GDI.150)
 0001:8344       UPDATELINKSDLGPROC
 0000:0000  Imp  UPDATEWINDOW         (USER.124)
 0001:9C80       USTANDARDHOOK
 0001:9ABC       USTANDARDINVOCATION
 0001:995C       USTANDARDVALIDATION
 0000:0000  Imp  WAITEVENT            (KERNEL.30)
 0001:2424       WINMAIN
 0000:0000  Imp  WRITECLASSSTG        (OLE2.19)
 0000:0000  Imp  WRITECLASSSTM        (OLE2.21)
 0000:0000  Imp  WRITEFMTUSERTYPESTG  (OLE2.75)
 0000:0000  Imp  WVSPRINTF            (USER.421)
 0001:9780       XFORMHEIGHTINHIMETRICTOPIXELS
 0000:0000  Unr  XFORMHEIGHTINPIXELSTOHIMETRIC
 0000:0000  Unr  XFORMRECTINHIMETRICTOPIXELS
 0001:97CC       XFORMRECTINPIXELSTOHIMETRIC
 0001:987C       XFORMSIZEINHIMETRICTOPIXELS
 0000:0000  Unr  XFORMSIZEINPIXELSTOHIMETRIC
 0001:9734       XFORMWIDTHINHIMETRICTOPIXELS
 0000:0000  Unr  XFORMWIDTHINPIXELSTOHIMETRIC
 0001:4058       _abort
 0003:08C2       _aseghi
 0003:08C0       _aseglo
 0001:3464       _atoi
 0003:1A52       _cfEmbeddedObject
 0003:1A50       _cfEmbedSource
 0003:1A5A       _cfFileName
 0003:1A5C       _cfLinkSource
 0003:1A58       _cfLinkSrcDescriptor
 0003:1A5E       _cfObjectDescriptor
 0003:1A56       _cfOwnerLink
 0003:0ED0       _edata
 0003:1A60       _end
 0003:0A18       _errno
 0001:3AD7       _exit
 0001:ABFA       _FChangeIconInit
 0001:502C       _fclose
 0001:B178       _FDrawListIcon
 0001:4E90       _fflush
 0001:B330       _FIconBoxInitialize
 0001:64F6       _FInsertObjectInit
 0001:BB2E       _FResultImageInitialize
 0001:6DC4       _FToggleObjectSource
 0001:74F8       _FValidateInsertFile
 0003:1A54       _ghInst
 0000:0000  Imp  _GUID_NULL           (COMPOBJ.37)
 0003:0848       _g_dwLockCount
 0003:0844       _g_dwObjectCount
 0001:B3A6       _IconBoxUninitialize
 0000:0000  Imp  _IID_IAdviseSink     (OLE2.135)
 0000:0000  Imp  _IID_IDataObject     (OLE2.134)
 0000:0000  Imp  _IID_IDropSource     (OLE2.153)
 0000:0000  Imp  _IID_IDropTarget     (OLE2.154)
 0000:0000  Imp  _IID_IEnumFORMATETC  (OLE2.123)
 0000:0000  Imp  _IID_IOleCache       (OLE2.150)
 0000:0000  Imp  _IID_IOleClientSite  (OLE2.144)
 0000:0000  Imp  _IID_IOleLink        (OLE2.149)
 0000:0000  Imp  _IID_IOleObject      (OLE2.138)
 0000:0000  Imp  _IID_IPersistStorage (OLE2.130)
 0000:0000  Imp  _IID_IUnknown        (COMPOBJ.38)
 0000:0000  Imp  _IID_IViewObject     (OLE2.133)
 0000:0000  Imp  _IID_IViewObject2    (OLE2.158)
 0001:7586       _InsertObjectCleanup
 0001:7900       _OleStdEnumFmtEtc_AddRef
 0001:7AC2       _OleStdEnumFmtEtc_Clone
 0001:77CE       _OleStdEnumFmtEtc_Destroy
 0001:795E       _OleStdEnumFmtEtc_Next
 0001:787A       _OleStdEnumFmtEtc_QueryInterface
 0001:7920       _OleStdEnumFmtEtc_Release
 0001:7AA8       _OleStdEnumFmtEtc_Reset
 0001:7A32       _OleStdEnumFmtEtc_Skip
 0001:9392       _OleStdNullMethod
 0000:0000  Unr  _OleUIPromptUser
 0001:527E       _remove
 0001:BC1E       _ResultImageUninitialize
 0001:72D6       _SetInsertObjectResults
 0001:407A       _sprintf
 0003:08B4       _STKHQQ
 0001:520E       _strcat
 0001:3FAC       _strcpy
 0001:3468       _strcspn
 0001:3FE8       _strlen
 0001:34C4       _strstr
 0001:353C       _strtol
 0001:3530       _strtoul
 0001:240C       _TestDebugOut
 0001:BDA0       _TransparentBlt
 0001:68F6       _UFillClassList
 0001:B01A       _UFillIconList
 0003:0850       _uMsgBrowse
 0003:0852       _uMsgChangeIcon
 0003:0856       _uMsgCloseBusyDlg
 0003:084E       _uMsgEndDialog
 0003:0854       _uMsgFileOKString
 0003:084C       _uMsgHelp
 0001:70B0       _UpdateClassIcon
 0001:7052       _UpdateClassType
 0001:B240       _UpdateResultIcon
 0000:0000  Imp  _wsprintf            (USER.420)
 0003:0AFE       __aaltstkovr
 0003:09FC       __acfinfo
 0000:9876  Abs  __acrtmsg
 0000:9876  Abs  __acrtused
 0000:D6D6  Abs  __aDBdoswp
 0003:0A6A       __adbgmsg
 0000:D6D6  Abs  __aDBused
 0001:4AD4       __aFchkstk
 0001:3894       __aFlmul
 0001:3894       __aFulmul
 0000:0000  Imp  __AHINCR             (KERNEL.114)
 0003:0A0A       __aintdiv
 0003:0AFC       __amblksiz
 0001:3E44       __amsg_exit
 0001:4AB4       __aNchkstk
 0003:0B24       __asizeC
 0003:0B25       __asizeD
 0001:366E       __assert
 0001:3384       __astart
 0001:4002       __catox
 0001:3AF4       __cexit
 0003:0B04       __cfltcvt_tab
 0003:0B26       __cflush
 0001:4190       __chdrive
 0003:0A67       __child
 0001:4AD4       __chkstk
 0001:39F4       __cinit
 0001:3E3A       __cintDIV
 0001:51D6       __close
 0001:52C8       __cltoasub
 0003:08BE       __cmdShow
 0001:512E       __commit
 0003:0A27       __cpumode
 0001:3B75       __ctermsub
 0003:08C8       __ctype
 0003:08C8       __ctype_
 0001:52D5       __cxtoa
 0001:3B05       __c_exit
 0003:0A28       __doserrno
 0001:3E86       __dosret0
 0001:3EA5       __dosretax
 0001:3E93       __dosreturn
 0001:52A4       __dos_commit
 0001:381A       __dos_findfirst
 0001:3808       __dos_findnext
 0003:0ED0       __edata
 0003:1A60       __end
 0001:4E66       __endstdio
 0003:0A5E       __environ
 0001:3AE5       __exit
 0003:0A69       __exitflag
 0003:0A0E       __fac
 0001:4FEC       __fcloseall
 0001:3EE4       __ffree
 0001:3BB2       __FF_MSGBANNER
 0003:0AEE       __fheap
 0001:4A11       __findlast
 0001:429E       __flsbuf
 0001:4EEC       __flush
 0001:4F6C       __flushall
 0001:3F05       __fmalloc
 0001:38C6       __fmemcmp
 0001:3922       __fmemcpy
 0001:3980       __fmemset
 0003:0B34       __fpinit
 0000:9876  Abs  __fptaskdata
 0001:41E6       __fptrap
 0001:36BC       __fpurecall
 0001:519E       __freebuf
 0001:4B22       __getbuf
 0001:36C2       __getcwd
 0001:36E0       __getdcwd
 0001:428E       __GetDGROUP
 0001:4166       __getdrive
 0001:491A       __growseg
 0003:08B8       __hInstance
 0003:08B6       __hPrevInstance
 0001:49AB       __incseg
 0001:4DFC       __initseg
 0001:40E8       __intdosx
 0003:0B44       __iob
 0003:0C34       __iob2
 0001:5262       __itoa
 0003:0B02       __lastiob
 0001:4E30       __linkseg
 0003:08BA       __lpszCmdLine
 0001:4B6E       __lseek
 0003:0B28       __lseekchk
 0001:3EB7       __maperror
 0001:4260       __myalloc
 0001:4A32       __newseg
 0003:0A2A       __nfile
 0001:41EC       __NMSG_TEXT
 0001:4223       __NMSG_WRITE
 0001:343B       __nomain
 0001:36BC       __npurecall
 0003:0A28       __oserr
 0003:0A30       __osfile
 0003:0A23       __osmajor
 0003:0A22       __osminor
 0003:0A26       __osmode
 0003:0A22       __osver
 0003:0A24       __osversion
 0001:43A8       __output
 0003:0A62       __pgmptr
 0003:0A86       __pnhFarHeap
 0003:0A1E       __psp
 0003:0A1C       __pspadr
 0001:36BC       __purecall
 0001:41DF       __QWINClose
 0001:41DF       __QWINExit
 0001:41DF       __QWINGetBuffSize
 0001:41DF       __QWINGetFocus
 0001:41DF       __QWINGetSize
 0001:41DF       __QWINInit
 0001:41DF       __QWINIsQWINin
 0001:41DF       __QWINMenuClick
 0001:41DF       __QWINOpen
 0001:41DF       __QWINRead
 0001:41DF       __QWINSetAboutString
 0001:41DF       __QWINSetBuffSize
 0001:41DF       __QWINSetFocus
 0001:41DF       __QWINSetSize
 0001:41DF       __QWINTerm
 0003:0A8A       __qwinused
 0001:41DF       __QWINWrite
 0001:41DF       __QWINYield
 0001:489E       __searchseg
 0001:3BD6       __setargv
 0001:3D80       __setenvp
 0003:0B22       __sigintoff
 0003:0B20       __sigintseg
 0000:0001  Abs  __sizec
 0000:0001  Abs  __sized
 0001:4E7C       __stackavail
 0001:39C8       __stubmain
 0003:0A1A       __umaskval
 0001:527E       __unlink
 0001:41DF       __wabout
 0001:41DA       __wcexit
 0001:41DA       __wcinit
 0001:41DF       __wclose
 0003:0A2C       __wfile
 0001:337A       __wflags
 0001:41DF       __wgetfocus
 0001:41DF       __wgetscreenbuf
 0001:41DF       __wgetsize
 0000:0000  Imp  __WINFLAGS           (KERNEL.178)
 0003:0A21       __winmajor
 0003:0A20       __winminor
 0003:0A20       __winver
 0000:0000  Abs  __wiobused
 0001:41DF       __wmenuclick
 0003:0A2E       __wnfile
 0001:41DF       __wopen
 0001:41DF       __wread
 0001:4C42       __write
 0001:41DF       __wsetfocus
 0001:41DF       __wsetscreenbuf
 0001:41DF       __wsetsize
 0003:0A44       __wsfile
 0001:41DF       __wterm
 0001:41DF       __wwrite
 0003:08C6       ___aDBrterr
 0003:08C4       ___aDBswpflg
 0003:0A58       ___argc
 0003:0A5A       ___argv
 0001:4B0E       ___ExportedStub

  Address         Publics by Value

 0000:0000  Imp  STRINGFROMCLSID      (COMPOBJ.19)
 0000:0000  Imp  GETMENUITEMCOUNT     (USER.263)
 0000:0000  Imp  OFFSETRECT           (USER.77)
 0000:0000  Imp  EXTRACTICON          (SHELL.34)
 0000:0000  Unr  HICONFROMCLASS
 0000:0000  Unr  XFORMRECTINHIMETRICTOPIXELS
 0000:0000  Imp  ENABLEMENUITEM       (USER.155)
 0000:0000  Imp  ENUMMETAFILE         (GDI.175)
 0000:0000  Imp  LSTRCMPI             (USER.471)
 0000:0000  Imp  LOADBITMAP           (USER.175)
 0000:0000  Imp  GETSYSCOLOR          (USER.180)
 0000:0000  Imp  FINDRESOURCE         (KERNEL.60)
 0000:0000  Imp  GETCLASSFILE         (OLE2.57)
 0000:0000  Unr  PARSECMDLINE
 0000:0000  Imp  REGISTERCLIPBOARDFORMAT (USER.145)
 0000:0000  Imp  RELEASESTGMEDIUM     (OLE2.32)
 0000:0000  Imp  CREATEIC             (GDI.153)
 0000:0000  Imp  CREATEDC             (GDI.53)
 0000:0000  Imp  RELEASEDC            (USER.68)
 0000:0000  Imp  GLOBALFREE           (KERNEL.17)
 0000:0000  Imp  REGISTERWINDOWMESSAGE (USER.118)
 0000:0000  Imp  SETBRUSHORG          (GDI.148)
 0000:0000  Imp  SETWINDOWORGEX       (GDI.482)
 0000:0000  Unr  OLESTDCREATETEMPFILEMONIKER
 0000:0000  Abs  __wiobused
 0000:0000  Unr  RESETORIGDC
 0000:0000  Imp  DESTROYMENU          (USER.152)
 0000:0000  Unr  OLESTDGETMISCSTATUSOFCLASS
 0000:0000  Imp  UPDATEWINDOW         (USER.124)
 0000:0000  Imp  DODRAGDROP           (OLE2.37)
 0000:0000  Imp  _IID_IDropSource     (OLE2.153)
 0000:0000  Unr  OLESTDDOTREATASCLASS
 0000:0000  Imp  SETMESSAGEQUEUE      (USER.266)
 0000:0000  Imp  GETWINDOWTEXT        (USER.36)
 0000:0000  Imp  SETWINDOWTEXT        (USER.37)
 0000:0000  Imp  SHOWWINDOW           (USER.42)
 0000:0000  Imp  PLAYMETAFILE         (GDI.123)
 0000:0000  Imp  ANSIPREV             (USER.473)
 0000:0000  Imp  PROGIDFROMCLSID      (COMPOBJ.62)
 0000:0000  Imp  DEFWINDOWPROC        (USER.107)
 0000:0000  Imp  _IID_IOleClientSite  (OLE2.144)
 0000:0000  Imp  MKPARSEDISPLAYNAME   (OLE2.23)
 0000:0000  Imp  _IID_IAdviseSink     (OLE2.135)
 0000:0000  Unr  OLESTDOPENCHILDSTORAGE
 0000:0000  Imp  OLEQUERYLINKFROMDATA (OLE2.6)
 0000:0000  Imp  GETPARENT            (USER.46)
 0000:0000  Imp  FATALEXIT            (KERNEL.1)
 0000:0000  Imp  OLEGETICONOFCLASS    (OLE2.53)
 0000:0000  Unr  OLESTDGETPRIORITYCLIPBOARDFORMAT
 0000:0000  Unr  OLESTDGETLINKSOURCEDATA
 0000:0000  Imp  CREATECOMPATIBLEBITMAP (GDI.51)
 0000:0000  Imp  _IID_IUnknown        (COMPOBJ.38)
 0000:0000  Imp  ISWINDOW             (USER.47)
 0000:0000  Imp  SETMAPMODE           (GDI.3)
 0000:0000  Imp  DIALOGBOXINDIRECTPARAM (USER.240)
 0000:0000  Imp  DISPATCHMESSAGE      (USER.114)
 0000:0000  Imp  CREATEICON           (USER.407)
 0000:0000  Unr  OLESTDSETICONINCACHE
 0000:0000  Imp  DELETEMETAFILE       (GDI.127)
 0000:0000  Imp  DRAWFOCUSRECT        (USER.466)
 0000:0000  Imp  DESTROYICON          (USER.457)
 0000:0000  Imp  DOS3CALL             (KERNEL.102)
 0000:0000  Imp  STGOPENSTORAGE       (STORAGE.3)
 0000:0000  Imp  WRITEFMTUSERTYPESTG  (OLE2.75)
 0000:0000  Imp  UNREALIZEOBJECT      (GDI.150)
 0000:0000  Imp  LOADRESOURCE         (KERNEL.61)
 0000:0000  Imp  ISBADCODEPTR         (KERNEL.336)
 0000:0000  Imp  FREEPROCINSTANCE     (KERNEL.52)
 0000:0000  Unr  OLESTDCREATEDC
 0000:0000  Imp  _IID_IDropTarget     (OLE2.154)
 0000:0000  Unr  OLESTDCREATEIC
 0000:0000  Unr  OLESTDMKPARSEDISPLAYNAME
 0000:0000  Imp  INSERTMENU           (USER.410)
 0000:0000  Imp  DELETEMENU           (USER.413)
 0000:0000  Imp  __WINFLAGS           (KERNEL.178)
 0000:0000  Unr  OLESTDOPENORCREATEROOTSTORAGE
 0000:0000  Imp  ISBADREADPTR         (KERNEL.334)
 0000:0000  Imp  OLEDUPLICATEDATA     (OLE2.51)
 0000:0000  Imp  COLOCKOBJECTEXTERNAL (COMPOBJ.63)
 0000:0000  Imp  WVSPRINTF            (USER.421)
 0000:0000  Imp  PTINRECT             (USER.76)
 0000:0000  Imp  POSTQUITMESSAGE      (USER.6)
 0000:0000  Imp  GETPROP              (USER.25)
 0000:0000  Imp  SETPROP              (USER.26)
 0000:0000  Imp  COISOLE1CLASS        (COMPOBJ.36)
 0000:0000  Imp  _IID_IEnumFORMATETC  (OLE2.123)
 0000:0000  Imp  LOCKRESOURCE         (KERNEL.62)
 0000:0000  Imp  REVOKEDRAGDROP       (OLE2.36)
 0000:0000  Imp  CREATEBINDCTX        (OLE2.26)
 0000:0000  Unr  OLESTDFILLOBJECTDESCRIPTORFROMDATA
 0000:0000  Imp  SETDLGITEMTEXT       (USER.92)
 0000:0000  Imp  GETDLGITEMTEXT       (USER.93)
 0000:0000  Imp  SENDDLGITEMMESSAGE   (USER.101)
 0000:0000  Unr  XFORMSIZEINPIXELSTOHIMETRIC
 0000:0000  Imp  SETDIBITS            (GDI.440)
 0000:0000  Imp  _IID_IViewObject2    (OLE2.158)
 0000:0000  Imp  READCLASSSTG         (OLE2.18)
 0000:0000  Imp  ISBADWRITEPTR        (KERNEL.335)
 0000:0000  Imp  GETDIALOGBASEUNITS   (USER.243)
 0000:0000  Imp  EXTTEXTOUT           (GDI.351)
 0000:0000  Imp  GETSYSTEMMETRICS     (USER.179)
 0000:0000  Imp  CLSIDFROMPROGID      (COMPOBJ.61)
 0000:0000  Imp  SETCURSOR            (USER.69)
 0000:0000  Imp  LOADCURSOR           (USER.173)
 0000:0000  Imp  REGISTERCLASS        (USER.57)
 0000:0000  Unr  OLESTDGETLENFILEPREFIXOFMONIKER
 0000:0000  Unr  UCLASSFROMDESCRIPTION
 0000:0000  Imp  LOADICON             (USER.174)
 0000:0000  Imp  ENDPAINT             (USER.40)
 0000:0000  Unr  OLESTDCOMMITSTORAGE
 0000:0000  Unr  OLESTDDOCONVERT
 0000:0000  Imp  SETTIMER             (USER.10)
 0000:0000  Unr  OLESTDCREATETARGETDEVICE
 0000:0000  Imp  LSTRCPYN             (KERNEL.353)
 0000:0000  Imp  OLECREATELINKTOFILE  (OLE2.68)
 0000:0000  Imp  CREATEPALETTE        (GDI.360)
 0000:0000  Imp  SENDMESSAGE          (USER.111)
 0000:0000  Unr  OLESTDDESTROYALLELEMENTS
 0000:0000  Imp  OLESAVE              (OLE2.13)
 0000:0000  Imp  FREERESOURCE         (KERNEL.63)
 0000:0000  Imp  CREATEFILEMONIKER    (OLE2.28)
 0000:0000  Imp  OLECREATEFROMFILE    (OLE2.67)
 0000:0000  Imp  STGCREATEDOCFILEONILOCKBYTES (STORAGE.2)
 0000:0000  Unr  OLESTDDELETETARGETDEVICE
 0000:0000  Imp  _IID_IOleObject      (OLE2.138)
 0000:0000  Imp  REGOPENKEY           (SHELL.1)
 0000:0000  Imp  PEEKMESSAGE          (USER.109)
 0000:0000  Imp  GETDLGITEM           (USER.91)
 0000:0000  Imp  SELECTPALETTE        (USER.282)
 0000:0000  Imp  SETBKCOLOR           (GDI.1)
 0000:0000  Imp  GETBKCOLOR           (GDI.75)
 0000:0000  Imp  OEMTOANSI            (KEYBOARD.6)
 0000:0000  Imp  CREATEHATCHBRUSH     (GDI.58)
 0000:0000  Imp  _IID_IDataObject     (OLE2.134)
 0000:0000  Imp  OLELOAD              (OLE2.12)
 0000:0000  Imp  CREATEFONTINDIRECT   (GDI.57)
 0000:0000  Imp  FILLRECT             (USER.81)
 0000:0000  Imp  RESTOREDC            (GDI.39)
 0000:0000  Imp  PLAYMETAFILERECORD   (GDI.176)
 0000:0000  Unr  OLEUICANUNLOADNOW
 0000:0000  Imp  ENDDIALOG            (USER.88)
 0000:0000  Imp  DIALOGBOXPARAM       (USER.239)
 0000:0000  Imp  REGCLOSEKEY          (SHELL.3)
 0000:0000  Unr  SETDCTOANISOTROPIC
 0000:0000  Imp  REALIZEPALETTE       (USER.283)
 0000:0000  Imp  OLEFLUSHCLIPBOARD    (OLE2.76)
 0000:0000  Imp  BITBLT               (GDI.34)
 0000:0000  Unr  OLESTDISDUPLICATEFORMAT
 0000:0000  Imp  REMOVEPROP           (USER.24)
 0000:0000  Imp  GETMESSAGE           (USER.108)
 0000:0000  Imp  COGETMALLOC          (COMPOBJ.4)
 0000:0000  Imp  OLESETCLIPBOARD      (OLE2.49)
 0000:0000  Imp  BRINGWINDOWTOTOP     (USER.45)
 0000:0000  Imp  OLECREATE            (OLE2.10)
 0000:0000  Unr  OLESTDNOTEFILECHANGETIME
 0000:0000  Unr  OLESTDCREATEROOTSTORAGE
 0000:0000  Imp  OLEINITIALIZE        (OLE2.2)
 0000:0000  Imp  GETSUBMENU           (USER.159)
 0000:0000  Imp  CREATESOLIDBRUSH     (GDI.66)
 0000:0000  Imp  GLOBALLOCK           (KERNEL.18)
 0000:0000  Imp  SETWINDOWEXTEX       (GDI.481)
 0000:0000  Unr  OLESTDCHECKVTBL
 0000:0000  Imp  GETDEVICECAPS        (GDI.80)
 0000:0000  Imp  OLEBUILDVERSION      (OLE2.1)
 0000:0000  Unr  OLESTDGETTREATASFMTUSERTYPE
 0000:0000  Imp  LOADLIBRARY          (KERNEL.95)
 0000:0000  Unr  UDESCRIPTIONFROMCLASS
 0000:0000  Imp  MOVEWINDOW           (USER.56)
 0000:0000  Imp  SCREENTOCLIENT       (USER.29)
 0000:0000  Imp  REGSETVALUE          (SHELL.5)
 0000:0000  Imp  STGCREATEDOCFILE     (STORAGE.1)
 0000:0000  Imp  OLESAVETOSTREAM      (OLE2.24)
 0000:0000  Imp  SELECTOBJECT         (GDI.45)
 0000:0000  Unr  OLESTDNOTEOBJECTCHANGETIME
 0000:0000  Imp  GETWINDOWWORD        (USER.133)
 0000:0000  Imp  SETWINDOWWORD        (USER.134)
 0000:0000  Unr  OLESTDOPENROOTSTORAGE
 0000:0000  Imp  CREATEBITMAP         (GDI.48)
 0000:0000  Imp  GETWINDOWRECT        (USER.32)
 0000:0000  Imp  GLOBALUNLOCK         (KERNEL.19)
 0000:0000  Imp  REMOVEMENU           (USER.412)
 0000:0000  Imp  _wsprintf            (USER.420)
 0000:0000  Imp  _GUID_NULL           (COMPOBJ.37)
 0000:0000  Imp  OLEGETICONOFFILE     (OLE2.52)
 0000:0000  Imp  CLOSEMETAFILE        (GDI.126)
 0000:0000  Imp  RECTANGLE            (GDI.27)
 0000:0000  Imp  WAITEVENT            (KERNEL.30)
 0000:0000  Unr  CHOPTEXT
 0000:0000  Imp  ISEQUALGUID          (COMPOBJ.18)
 0000:0000  Unr  OLESTDREGISTERASRUNNING
 0000:0000  Imp  GETRUNNINGOBJECTTABLE (OLE2.30)
 0000:0000  Imp  CHECKDLGBUTTON       (USER.97)
 0000:0000  Imp  DELETEDC             (GDI.68)
 0000:0000  Imp  CREATEILOCKBYTESONHGLOBAL (OLE2.54)
 0000:0000  Imp  GETCURRENTTIME       (USER.15)
 0000:0000  Imp  CREATECOMPATIBLEDC   (GDI.52)
 0000:0000  Imp  OLEMETAFILEPICTFROMICONANDLABEL (OLE2.56)
 0000:0000  Imp  DESTROYWINDOW        (USER.53)
 0000:0000  Imp  CODOSDATETIMETOFILETIME (COMPOBJ.31)
 0000:0000  Imp  INVALIDATERECT       (USER.125)
 0000:0000  Imp  _IID_IOleCache       (OLE2.150)
 0000:0000  Imp  OLEUNINITIALIZE      (OLE2.3)
 0000:0000  Imp  LSTRLEN              (KERNEL.90)
 0000:0000  Unr  OLESTDSETUPADVISES
 0000:0000  Imp  BEGINPAINT           (USER.39)
 0000:0000  Imp  GETFOCUS             (USER.23)
 0000:0000  Imp  FATALAPPEXIT         (KERNEL.137)
 0000:0000  Imp  SETROP2              (GDI.4)
 0000:0000  Imp  SETCONVERTSTG        (OLE2.83)
 0000:0000  Unr  XFORMWIDTHINPIXELSTOHIMETRIC
 0000:0000  Imp  CHECKRADIOBUTTON     (USER.96)
 0000:0000  Imp  DELETEOBJECT         (GDI.69)
 0000:0000  Imp  FREELIBRARY          (KERNEL.96)
 0000:0000  Imp  _IID_IOleLink        (OLE2.149)
 0000:0000  Imp  OLECREATEFROMDATA    (OLE2.8)
 0000:0000  Unr  SETDCTODRAWINHIMETRICRECT
 0000:0000  Imp  CLSIDFROMSTRING      (COMPOBJ.20)
 0000:0000  Imp  SETFOCUS             (USER.22)
 0000:0000  Imp  _IID_IViewObject     (OLE2.133)
 0000:0000  Imp  ANSINEXT             (USER.472)
 0000:0000  Imp  COFILETIMENOW        (COMPOBJ.82)
 0000:0000  Imp  READFMTUSERTYPESTG   (OLE2.74)
 0000:0000  Imp  ISDLGBUTTONCHECKED   (USER.98)
 0000:0000  Imp  SETVIEWPORTORGEX     (GDI.480)
 0000:0000  Unr  HICONANDSOURCEFROMCLASS
 0000:0000  Imp  GETCLIENTRECT        (USER.33)
 0000:0000  Imp  OUTPUTDEBUGSTRING    (KERNEL.115)
 0000:0000  Imp  INFLATERECT          (USER.78)
 0000:0000  Imp  GETVERSION           (KERNEL.3)
 0000:0000  Imp  WRITECLASSSTG        (OLE2.19)
 0000:0000  Imp  GETTEXTEXTENTPOINT   (GDI.471)
 0000:0000  Imp  SETTEXTCOLOR         (GDI.9)
 0000:0000  Imp  MULDIV               (GDI.128)
 0000:0000  Unr  FSERVERFROMCLASS
 0000:0000  Imp  SETVIEWPORTEXTEX     (GDI.479)
 0000:0000  Imp  TRANSLATEMESSAGE     (USER.113)
 0000:0000  Imp  GETOBJECT            (GDI.82)
 0000:0000  Imp  GETMENU              (USER.157)
 0000:0000  Imp  INITAPP              (USER.5)
 0000:0000  Imp  LOCKSEGMENT          (KERNEL.23)
 0000:0000  Unr  OLESTDGETITEMTOKEN
 0000:0000  Unr  OLESTDISOLELINK
 0000:0000  Unr  OLESTDREVOKEASRUNNING
 0000:0000  Imp  GETSTOCKOBJECT       (GDI.87)
 0000:0000  Imp  RELEASECAPTURE       (USER.19)
 0000:0000  Imp  __AHINCR             (KERNEL.114)
 0000:0000  Unr  OLEUIUPDATELINKS
 0000:0000  Imp  LSTRCMP              (USER.430)
 0000:0000  Imp  OLEQUERYCREATEFROMDATA (OLE2.7)
 0000:0000  Imp  GETPROCADDRESS       (KERNEL.50)
 0000:0000  Imp  GETDC                (USER.66)
 0000:0000  Imp  LSTRCAT              (KERNEL.89)
 0000:0000  Imp  WRITECLASSSTM        (OLE2.21)
 0000:0000  Unr  _OleUIPromptUser
 0000:0000  Imp  ISDBCSLEADBYTE       (KERNEL.207)
 0000:0000  Imp  REGISTERDRAGDROP     (OLE2.35)
 0000:0000  Imp  OPENFILE             (KERNEL.74)
 0000:0000  Imp  LSTRCPY              (KERNEL.88)
 0000:0000  Imp  SETWINDOWPOS         (USER.232)
 0000:0000  Imp  OLEDRAW              (OLE2.58)
 0000:0000  Imp  GETDOSENVIRONMENT    (KERNEL.131)
 0000:0000  Unr  OLESTDCREATECHILDSTORAGE
 0000:0000  Imp  CREATEWINDOW         (USER.41)
 0000:0000  Imp  GLOBALSIZE           (KERNEL.20)
 0000:0000  Imp  GLOBALALLOC          (KERNEL.15)
 0000:0000  Imp  REGENUMKEY           (SHELL.7)
 0000:0000  Imp  DRAWICON             (USER.84)
 0000:0000  Unr  OLESTDICONLABELTEXTOUT
 0000:0000  Imp  MESSAGEBOX           (USER.1)
 0000:0000  Imp  OLESETCONTAINEDOBJECT (OLE2.86)
 0000:0000  Imp  GETPROFILEINT        (KERNEL.57)
 0000:0000  Imp  GETBITMAPBITS        (GDI.74)
 0000:0000  Imp  GETMODULEFILENAME    (KERNEL.49)
 0000:0000  Imp  DIALOGBOX            (USER.87)
 0000:0000  Imp  COTREATASCLASS       (COMPOBJ.66)
 0000:0000  Imp  MAKEPROCINSTANCE     (KERNEL.51)
 0000:0000  Unr  OLESTDSWITCHDISPLAYASPECT
 0000:0000  Unr  OLESTDINITVTBL
 0000:0000  Imp  CREATEPEN            (GDI.61)
 0000:0000  Imp  ANSITOOEM            (KEYBOARD.5)
 0000:0000  Imp  SHOWCURSOR           (USER.71)
 0000:0000  Imp  ENABLEWINDOW         (USER.34)
 0000:0000  Imp  KILLTIMER            (USER.12)
 0000:0000  Imp  _IID_IPersistStorage (OLE2.130)
 0000:0000  Imp  CREATESTREAMONHGLOBAL (OLE2.84)
 0000:0000  Unr  XFORMHEIGHTINPIXELSTOHIMETRIC
 0000:0000  Imp  INITTASK             (KERNEL.91)
 0000:0000  Imp  LOADSTRING           (USER.176)
 0000:0000  Imp  CREATEMETAFILE       (GDI.125)
 0000:0000  Unr  OLESTDREALLOC
 0000:0000  Imp  GLOBALREALLOC        (KERNEL.16)
 0000:0000  Imp  CREATEPOPUPMENU      (USER.415)
 0000:0000  Imp  REGQUERYVALUE        (SHELL.6)
 0000:0000  Unr  OLESTDGETSIZE
 0000:0000  Imp  SETCAPTURE           (USER.18)
 0000:0000  Imp  SAVEDC               (GDI.30)
 0000:0000  Imp  ISDIALOGMESSAGE      (USER.90)
 0000:0000  Unr  OLESTDGETAUXUSERTYPE
 0000:0000  Imp  POSTMESSAGE          (USER.110)
 0000:0001  Abs  __sizec
 0000:0001  Abs  __sized
 0000:0006  Abs  pLocalHeap
 0000:0008  Abs  pAtomTable
 0000:000A  Abs  pStackTop
 0000:000C  Abs  pStackMin
 0000:000E  Abs  pStackBot
 0000:9876  Abs  __acrtused
 0000:9876  Abs  __fptaskdata
 0000:9876  Abs  __acrtmsg
 0000:D6D6  Abs  __aDBused
 0000:D6D6  Abs  __aDBdoswp
 0001:0000       ??0CSimpleApp@@REC@XZ
 0001:0052       ??1CSimpleApp@@REC@XZ
 0001:0082       ?DestroyDocs@CSimpleApp@@RECXXZ
 0001:009A       ?QueryInterface@CSimpleApp@@VEAPEXAFUGUID@@PEPEX@Z
 0001:00C4       ?AddRef@CSimpleApp@@VEAKXZ
 0001:00E8       ?Release@CSimpleApp@@VEAKXZ
 0001:0134       ?fInitApplication@CSimpleApp@@RECHI@Z
 0001:01F0       ?fInitInstance@CSimpleApp@@RECHIH@Z
 0001:02FE       ?lCommandHandler@CSimpleApp@@RECJIIIJ@Z
 0001:0448       ?lSizeHandler@CSimpleApp@@RECJIIIJ@Z
 0001:0476       ?lCreateDoc@CSimpleApp@@RECJIIIJ@Z
 0001:04AC       ?HandleAccelerators@CSimpleApp@@RECHPEUtagMSG@@@Z
 0001:04B2       ?PaintApp@CSimpleApp@@RECXI@Z
 0001:04D6       ?Create@CSimpleDoc@@TAPEV1@PEVCSimpleApp@@PEUtagRECT@@I@Z
 0001:0602       ?Close@CSimpleDoc@@RECXXZ
 0001:0672       ??0CSimpleDoc@@REC@PEVCSimpleApp@@I@Z
 0001:07A0       ??1CSimpleDoc@@REC@XZ
 0001:08D8       ?QueryInterface@CSimpleDoc@@VEAPEXAFUGUID@@PEPEX@Z
 0001:09AC       ?AddRef@CSimpleDoc@@VEAKXZ
 0001:09D0       ?Release@CSimpleDoc@@VEAKXZ
 0001:0A1C       ?InsertObject@CSimpleDoc@@RECXXZ
 0001:0B5C       ?lResizeDoc@CSimpleDoc@@RECJPEUtagRECT@@@Z
 0001:0B86       ?lAddVerbs@CSimpleDoc@@RECJXZ
 0001:0BEE       ?PaintDoc@CSimpleDoc@@RECXI@Z
 0001:0C12       ?DisableInsertObject@CSimpleDoc@@RECXXZ
 0001:0C60       ?CopyObjectToClip@CSimpleDoc@@RECXXZ
 0001:0D68       ?Create@CDataXferObj@@TAPEV1@PEVCSimpleSite@@PEUtagPOINTL@@@Z
 0001:0F54       ??0CDataXferObj@@BEC@XZ
 0001:0FC2       ??1CDataXferObj@@BEC@XZ
 0001:1032       ?QueryInterface@CDataXferObj@@VEAPEXAFUGUID@@PEPEX@Z
 0001:10B6       ?AddRef@CDataXferObj@@VEAKXZ
 0001:10DA       ?Release@CDataXferObj@@VEAKXZ
 0001:1126       ?QueryGetData@CDataXferObj@@VEAPEXPEUtagFORMATETC@@@Z
 0001:11C8       ?EnumFormatEtc@CDataXferObj@@VEAPEXKPEPEUIEnumFORMATETC@@@Z
 0001:123C       ?GetData@CDataXferObj@@VEAPEXPEUtagFORMATETC@@PEUtagSTGMEDIUM@@@Z
 0001:1402       ?GetDataHere@CDataXferObj@@VEAPEXPEUtagFORMATETC@@PEUtagSTGMEDIUM@@@Z
 0001:14E4       ?QueryInterface@CAdviseSink@@VEAPEXAFUGUID@@PEPEX@Z
 0001:1520       ?AddRef@CAdviseSink@@VEAKXZ
 0001:1554       ?Release@CAdviseSink@@VEAKXZ
 0001:1588       ?OnDataChange@CAdviseSink@@VEAXPEUtagFORMATETC@@PEUtagSTGMEDIUM@@@Z
 0001:15A0       ?OnViewChange@CAdviseSink@@VEAXKJ@Z
 0001:163E       ?OnRename@CAdviseSink@@VEAXPEUIMoniker@@@Z
 0001:1656       ?OnSave@CAdviseSink@@VEAXXZ
 0001:166E       ?OnClose@CAdviseSink@@VEAXXZ
 0001:1686       ?QueryDrag@CSimpleDoc@@RECHUtagPOINT@@@Z
 0001:16C8       ?DoDragDrop@CSimpleDoc@@RECKXZ
 0001:1792       ?QueryInterface@CDropSource@@VEAPEXAFUGUID@@PEPEX@Z
 0001:17CE       ?AddRef@CDropSource@@VEAKXZ
 0001:1802       ?Release@CDropSource@@VEAKXZ
 0001:1836       ?QueryContinueDrag@CDropSource@@VEAPEXHK@Z
 0001:185E       ?GiveFeedback@CDropSource@@VEAPEXK@Z
 0001:1870       ?QueryDrop@CDropTarget@@BECHKUtagPOINTL@@HPEK@Z
 0001:19B6       ?DoDragScroll@CDropTarget@@BECHUtagPOINTL@@@Z
 0001:1C3C       ?InitDragFeedback@CDropTarget@@BECXPEUIDataObject@@UtagPOINTL@@@Z
 0001:1D5C       ?UndrawDragFeedback@CDropTarget@@BECXXZ
 0001:1DB8       ?DrawDragFeedback@CDropTarget@@BECXUtagPOINTL@@@Z
 0001:1E7E       ?QueryInterface@CDropTarget@@VEAPEXAFUGUID@@PEPEX@Z
 0001:1EBA       ?AddRef@CDropTarget@@VEAKXZ
 0001:1EEE       ?Release@CDropTarget@@VEAKXZ
 0001:1F22       ?DragEnter@CDropTarget@@VEAPEXPEUIDataObject@@KUtagPOINTL@@PEK@Z
 0001:1FD6       ?DragOver@CDropTarget@@VEAPEXKUtagPOINTL@@PEK@Z
 0001:2050       ?DragLeave@CDropTarget@@VEAPEXXZ
 0001:2074       ?Drop@CDropTarget@@VEAPEXPEUIDataObject@@KUtagPOINTL@@PEK@Z
 0001:21C6       ?QueryInterface@COleClientSite@@VEAPEXAFUGUID@@PEPEX@Z
 0001:2202       ?AddRef@COleClientSite@@VEAKXZ
 0001:2236       ?Release@COleClientSite@@VEAKXZ
 0001:226A       ?SaveObject@COleClientSite@@VEAPEXXZ
 0001:2310       ?GetMoniker@COleClientSite@@VEAPEXKKPEPEUIMoniker@@@Z
 0001:233A       ?GetContainer@COleClientSite@@VEAPEXPEPEUIOleContainer@@@Z
 0001:2364       ?ShowObject@COleClientSite@@VEAPEXXZ
 0001:237E       ?OnShowWindow@COleClientSite@@VEAPEXH@Z
 0001:23EE       ?RequestNewObjectLayout@COleClientSite@@VEAPEXXZ
 0001:240C       _TestDebugOut
 0001:2424       WINMAIN
 0001:2566       ?MainWndProc@@ZCJIIIJ@Z
 0001:267A       ?About@@ZCHIIGJ@Z
 0001:26B2       ?DocWndProc@@ZCJIIIJ@Z
 0001:28FE       ?Create@CSimpleSite@@TAPEV1@PEVCSimpleDoc@@@Z
 0001:29BE       ??0CSimpleSite@@REC@PEVCSimpleDoc@@@Z
 0001:2AB8       ??1CSimpleSite@@REC@XZ
 0001:2B98       ?CloseOleObject@CSimpleSite@@RECXXZ
 0001:2BD0       ?UnloadOleObject@CSimpleSite@@RECXXZ
 0001:2C7A       ?QueryInterface@CSimpleSite@@VEAPEXAFUGUID@@PEPEX@Z
 0001:2D4E       ?AddRef@CSimpleSite@@VEAKXZ
 0001:2D72       ?Release@CSimpleSite@@VEAKXZ
 0001:2DBE       ?InitObject@CSimpleSite@@RECPEXH@Z
 0001:2F4E       ?PaintObj@CSimpleSite@@RECXI@Z
 0001:30BA       ?GetObjRect@CSimpleSite@@RECXPEUtagRECT@@@Z
 0001:30F6       ?StartTest1@@ZAXPEVCSimpleApp@@@Z
 0001:3208       ?StartTest2@@ZAXPEVCSimpleApp@@@Z
 0001:337A       __wflags
 0001:3384       __astart
 0001:343B       __nomain
 0001:3442       ??3@ZAXPEX@Z
 0001:3454       ??2@ZAPEXI@Z
 0001:3464       _atoi
 0001:3468       _strcspn
 0001:34C4       _strstr
 0001:3530       _strtoul
 0001:353C       _strtol
 0001:366E       __assert
 0001:36BC       __fpurecall
 0001:36BC       __purecall
 0001:36BC       __npurecall
 0001:36C2       __getcwd
 0001:36E0       __getdcwd
 0001:3808       __dos_findnext
 0001:381A       __dos_findfirst
 0001:3894       __aFulmul
 0001:3894       __aFlmul
 0001:38C6       __fmemcmp
 0001:3922       __fmemcpy
 0001:3980       __fmemset
 0001:39C8       __stubmain
 0001:39F4       __cinit
 0001:3AD7       _exit
 0001:3AE5       __exit
 0001:3AF4       __cexit
 0001:3B05       __c_exit
 0001:3B75       __ctermsub
 0001:3BB2       __FF_MSGBANNER
 0001:3BD6       __setargv
 0001:3D80       __setenvp
 0001:3E3A       __cintDIV
 0001:3E44       __amsg_exit
 0001:3E86       __dosret0
 0001:3E93       __dosreturn
 0001:3EA5       __dosretax
 0001:3EB7       __maperror
 0001:3EE4       __ffree
 0001:3F05       __fmalloc
 0001:3FAC       _strcpy
 0001:3FE8       _strlen
 0001:4002       __catox
 0001:4058       _abort
 0001:407A       _sprintf
 0001:40E8       __intdosx
 0001:4166       __getdrive
 0001:4190       __chdrive
 0001:41DA       __wcexit
 0001:41DA       __wcinit
 0001:41DF       __QWINOpen
 0001:41DF       __QWINSetSize
 0001:41DF       __QWINRead
 0001:41DF       __wsetscreenbuf
 0001:41DF       __wmenuclick
 0001:41DF       __wread
 0001:41DF       __QWINSetAboutString
 0001:41DF       __wsetsize
 0001:41DF       __wgetscreenbuf
 0001:41DF       __QWINExit
 0001:41DF       __wwrite
 0001:41DF       __QWINGetBuffSize
 0001:41DF       __QWINIsQWINin
 0001:41DF       __QWINSetBuffSize
 0001:41DF       __QWINWrite
 0001:41DF       __QWINYield
 0001:41DF       __QWINMenuClick
 0001:41DF       __wterm
 0001:41DF       __QWINSetFocus
 0001:41DF       __QWINGetFocus
 0001:41DF       __wabout
 0001:41DF       __QWINGetSize
 0001:41DF       __QWINInit
 0001:41DF       __wclose
 0001:41DF       __QWINTerm
 0001:41DF       __QWINClose
 0001:41DF       __wopen
 0001:41DF       __wsetfocus
 0001:41DF       __wgetfocus
 0001:41DF       __wgetsize
 0001:41E6       __fptrap
 0001:41EC       __NMSG_TEXT
 0001:4223       __NMSG_WRITE
 0001:4260       __myalloc
 0001:428E       __GetDGROUP
 0001:429E       __flsbuf
 0001:43A8       __output
 0001:489E       __searchseg
 0001:491A       __growseg
 0001:49AB       __incseg
 0001:4A11       __findlast
 0001:4A32       __newseg
 0001:4AB4       __aNchkstk
 0001:4AD4       __aFchkstk
 0001:4AD4       __chkstk
 0001:4B0E       ___ExportedStub
 0001:4B22       __getbuf
 0001:4B6E       __lseek
 0001:4C42       __write
 0001:4DFC       __initseg
 0001:4E30       __linkseg
 0001:4E66       __endstdio
 0001:4E7C       __stackavail
 0001:4E90       _fflush
 0001:4EEC       __flush
 0001:4F6C       __flushall
 0001:4FEC       __fcloseall
 0001:502C       _fclose
 0001:512E       __commit
 0001:519E       __freebuf
 0001:51D6       __close
 0001:520E       _strcat
 0001:5262       __itoa
 0001:527E       _remove
 0001:527E       __unlink
 0001:52A4       __dos_commit
 0001:52C8       __cltoasub
 0001:52D5       __cxtoa
 0001:5330       ??_7IUnknown@@6F@
 0001:533C       ??_7CSimpleApp@@6F@
 0001:5348       ?DAdvise@CDataXferObj@@VEAPEXPEUtagFORMATETC@@KPEUIAdviseSink@@PEK@Z
 0001:535A       ?DUnadvise@CDataXferObj@@VEAPEXK@Z
 0001:536C       ?EnumDAdvise@CDataXferObj@@VEAPEXPEPEUIEnumSTATDATA@@@Z
 0001:537E       ?GetCanonicalFormatEtc@CDataXferObj@@VEAPEXPEUtagFORMATETC@@0@Z
 0001:539C       ?SetData@CDataXferObj@@VEAPEXPEUtagFORMATETC@@PEUtagSTGMEDIUM@@H@Z
 0001:53AE       ??0CDropTarget@@REC@PEVCSimpleDoc@@@Z
 0001:542A       ??_C@_0O@GKMD@m_nCount?5?$DN?$DN?50?$AA@
 0001:5438       ??_C@_0BH@FLKL@In?5IDT?8s?5constructor?$AN?6?$AA@
 0001:5450       ??_C@_0BG@NDHK@In?5IDT?8s?5destructor?$AN?6?$AA@
 0001:5466       ??_C@_05NNFA@idt?4h?$AA@
 0001:546C       ??_C@_0BH@JHEO@In?5IDS?8s?5constructor?$AN?6?$AA@
 0001:5484       ??_C@_0BG@DGDH@In?5IDS?8s?5destructor?$AN?6?$AA@
 0001:549A       ??_7IDropTarget@@6F@
 0001:54B6       ??_7CSimpleDoc@@6F@
 0001:54C2       ??_7IDropSource@@6F@
 0001:54D6       ??_7CDropSource@@6F@
 0001:54EA       ??_7CDropTarget@@6F@
 0001:5506       ??_7CDataXferObj@@6F@
 0001:5536       ??_7IDataObject@@6F@
 0001:5566       ??_C@_0BI@IJIM@In?5IOCS?8s?5constructor?$AN?6?$AA@
 0001:557E       ??_C@_0BH@PEFE@In?5IOCS?8s?5destructor?$AN?6?$AA@
 0001:5596       ??_C@_06LNPM@iocs?4h?$AA@
 0001:559E       ??_C@_0BH@NFGK@In?5IAS?8s?5constructor?$AN?6?$AA@
 0001:55B6       ??_C@_0BG@BCJB@In?5IAS?8s?5destructor?$AN?6?$AA@
 0001:55CC       ??_C@_05NDCL@ias?4h?$AA@
 0001:55D2       ??_7COleClientSite@@6F@
 0001:55F6       ??_7IAdviseSink@@6F@
 0001:5616       ??_7IOleClientSite@@6F@
 0001:563A       ??_7CAdviseSink@@6F@
 0001:565A       ??_7CSimpleSite@@6F@
 0001:5666       OLEUIINSERTOBJECT
 0001:598C       INSERTOBJECTDIALOGPROC
 0001:64F6       _FInsertObjectInit
 0001:68F6       _UFillClassList
 0001:6DC4       _FToggleObjectSource
 0001:7052       _UpdateClassType
 0001:70B0       _UpdateClassIcon
 0001:72D6       _SetInsertObjectResults
 0001:74F8       _FValidateInsertFile
 0001:7586       _InsertObjectCleanup
 0001:75D2       ??_C@_0M@LNGB@COMMDLG?4DLL?$AA@
 0001:75DE       ??_C@_0N@PNI@GetFileTitle?$AA@
 0001:75EC       ??_C@_01PCFE@?2?$AA@
 0001:75EE       ??_C@_0CH@JMMM@?$CK?$CK?$CK?5Please?5install?5VC?$CL?$CL?5Patch?5?$CD1@
 0001:7616       ??_C@_0N@IIFK@commdlg_help?$AA@
 0001:7624       ??_C@_0P@PDBJ@?2NotInsertable?$AA@
 0001:7634       ??_C@_0CA@PANP@?2protocol?2StdFileEditing?2server?$AA@
 0001:7654       ??_C@_0M@PKFG@?2Insertable?$AA@
 0001:7660       ??_C@_06JPNA@?2CLSID?$AA@
 0001:7668       ??_C@_06HFAC@CLSID?2?$AA@
 0001:7670       ??_C@_0N@OIGG@?2LocalServer?$AA@
 0001:767E       ??_C@_0O@JEDJ@?2InProcServer?$AA@
 0001:768C       ??_C@_01POCP@?7?$AA@
 0001:768E       OLESTDENUMFMTETC_CREATE
 0001:77CE       _OleStdEnumFmtEtc_Destroy
 0001:787A       _OleStdEnumFmtEtc_QueryInterface
 0001:7900       _OleStdEnumFmtEtc_AddRef
 0001:7920       _OleStdEnumFmtEtc_Release
 0001:795E       _OleStdEnumFmtEtc_Next
 0001:7A32       _OleStdEnumFmtEtc_Skip
 0001:7AA8       _OleStdEnumFmtEtc_Reset
 0001:7AC2       _OleStdEnumFmtEtc_Clone
 0001:7B38       OLEUIINITIALIZE
 0001:7CBC       OLEUIUNINITIALIZE
 0001:7CD4       OLEUIADDVERBMENU
 0001:829E       PROMPTUSERDLGPROC
 0001:8344       UPDATELINKSDLGPROC
 0001:86C2       ??_C@_0N@OCMF@VERIFICATION?$AA@
 0001:86D0       ??_C@_0P@LMIA@OLEUI_MSG_HELP?$AA@
 0001:86E0       ??_C@_0BE@FEHN@OLEUI_MSG_ENDDIALOG?$AA@
 0001:86F4       ??_C@_0BB@PGGH@OLEUI_MSG_BROWSE?$AA@
 0001:8706       ??_C@_0BF@COIE@OLEUI_MSG_CHANGEICON?$AA@
 0001:871C       ??_C@_0BD@HNAP@commdlg_FileNameOK?$AA@
 0001:8730       ??_C@_0BK@LOCD@OLEUI_MSG_CLOSEBUSYDIALOG?$AA@
 0001:874A       ??_C@_0BC@GMEI@Object?5Descriptor?$AA@
 0001:875C       ??_C@_0BH@FOOO@Link?5Source?5Descriptor?$AA@
 0001:8774       ??_C@_0N@LHIH@Embed?5Source?$AA@
 0001:8782       ??_C@_0BA@IEJA@Embedded?5Object?$AA@
 0001:8792       ??_C@_0M@KPGD@Link?5Source?$AA@
 0001:879E       ??_C@_09NJ@OwnerLink?$AA@
 0001:87A8       ??_C@_08NJLM@FileName?$AA@
 0001:87B2       ??_C@_0M@MBIN@ole2uiRICls?$AA@
 0001:87BE       ??_C@_0M@GHPL@ole2uiIBCls?$AA@
 0001:87CA       ??_C@_0CG@HCKA@resource?5read?50x?$CFX?0?5my?5value?5is?5@
 0001:87F0       ??_C@_00A@?$AA@
 0001:87F2       ??_C@_03NAME@?4?4?4?$AA@
 0001:87F6       ??_C@_09DKHB@Structure?$AA@
 0001:8800       ??_C@_04FOAE@?$CFd?$CF?$CF?$AA@
 0001:8806       OLESTDQUERYINTERFACE
 0001:8844       OLESTDGETDATA
 0001:8940       OLESTDMALLOC
 0001:899E       OLESTDFREE
 0001:89F4       OLESTDFREESTRING
 0001:8A4A       OLESTDCOPYSTRING
 0001:8AD4       OLESTDCREATESTORAGEONHGLOBAL
 0001:8B6C       OLESTDCREATETEMPSTORAGE
 0001:8BCA       OLESTDGETOLEOBJECTDATA
 0001:8CD4       OLESTDGETOBJECTDESCRIPTORDATA
 0001:8E5A       OLESTDGETOBJECTDESCRIPTORDATAFROMOLEOBJECT
 0001:91D6       OLESTDGETMETAFILEPICTFROMOLEOBJECT
 0001:934A       OLESTDVERIFYRELEASE
 0001:936E       OLESTDRELEASE
 0001:9392       _OleStdNullMethod
 0001:9416       OLESTDGETFIRSTMONIKER
 0001:94CC       OLESTDMARKPASTEENTRYLIST
 0001:9676       ??_C@_0DJ@NHNH@OleStdSwitchDisplayAspect?3?5Cache@
 0001:96B0       ??_C@_05FGFK@CLSID?$AA@
 0001:96B6       ??_C@_09JJAI@Linked?5?$CFs?$AA@
 0001:96C0       ??_C@_07CPIP@Package?$AA@
 0001:96C8       ??_C@_0CL@HONB@ERROR?3?5INTERFACE?5METHOD?5NOT?5IMPL@
 0001:96F4       ??_C@_04MOFI@?$CFs?$CFd?$AA@
 0001:96FA       ??_C@_0DC@GEMK@OleStdCreateTempFileMoniker?3?5Mon@
 0001:972C       ??_C@_06KAHL@?$EA?$CFs?$CB?$CFs?$AA@
 0001:9734       XFORMWIDTHINHIMETRICTOPIXELS
 0001:9780       XFORMHEIGHTINHIMETRICTOPIXELS
 0001:97CC       XFORMRECTINPIXELSTOHIMETRIC
 0001:987C       XFORMSIZEINHIMETRICTOPIXELS
 0001:9952       ??_C@_09LHIP@Embedding?$AA@
 0001:995C       USTANDARDVALIDATION
 0001:9ABC       USTANDARDINVOCATION
 0001:9B4A       LPVSTANDARDINIT
 0001:9C08       LPVSTANDARDENTRY
 0001:9C80       USTANDARDHOOK
 0001:9CC4       STANDARDCLEANUP
 0001:9D14       STANDARDSHOWDLGITEM
 0001:9D6A       ??_C@_04CLJC@Font?$AA@
 0001:9D70       OLEUIMETAFILEPICTICONFREE
 0001:9DB8       OLEUIMETAFILEPICTICONDRAW
 0001:9ECC       ENUMMETAFILEICONDRAW
 0001:9F48       OLEUIMETAFILEPICTEXTRACTLABEL
 0001:A000       ENUMMETAFILEEXTRACTLABEL
 0001:A0DE       OLEUIMETAFILEPICTEXTRACTICON
 0001:A142       ENUMMETAFILEEXTRACTICON
 0001:A36E       OLEUIMETAFILEPICTEXTRACTICONSOURCE
 0001:A412       ENUMMETAFILEEXTRACTICONSOURCE
 0001:A518       OLEUICHANGEICON
 0001:A5BA       CHANGEICONDIALOGPROC
 0001:ABFA       _FChangeIconInit
 0001:B01A       _UFillIconList
 0001:B178       _FDrawListIcon
 0001:B240       _UpdateResultIcon
 0001:B324       ??_C@_0L@CPGB@HWND_CIDLG?$AA@
 0001:B330       _FIconBoxInitialize
 0001:B3A6       _IconBoxUninitialize
 0001:B3A8       ICONBOXWNDPROC
 0001:B532       OLESTDCOPYTARGETDEVICE
 0001:B584       OLESTDCOPYFORMATETC
 0001:B622       OLESTDCOMPAREFORMATETC
 0001:B6F0       OLESTDCOMPARETARGETDEVICE
 0001:B75A       ??_C@_07LGIJ@DISPLAY?$AA@
 0001:B884       OLESTDGETUSERTYPEOFCLASS
 0001:BA08       OLESTDGETDEFAULTFILEFORMATOFCLASS
 0001:BAE6       ??_C@_08BJKM@CLSID?2?$CFs?$AA@
 0001:BAF0       ??_C@_0BA@LJEI@?2AuxUserType?2?$CFd?$AA@
 0001:BB00       ??_C@_0M@BODG@?2MiscStatus?$AA@
 0001:BB0C       ??_C@_0CB@FCAE@CLSID?2?$CFs?2DataFormats?2DefaultFile@
 0001:BB2E       _FResultImageInitialize
 0001:BC1E       _ResultImageUninitialize
 0001:BC30       RESULTIMAGEWNDPROC
 0001:BDA0       _TransparentBlt
 0001:BF2A       HOURGLASSON
 0001:BF4A       HOURGLASSOFF
 0001:BF60       BROWSE
 0001:C0CE       REPLACECHARWITHNULL
 0001:C104       ERRORWITHFILE
 0001:C200       OPENFILEERROR
 0001:C5AE       DOESFILEEXIST
 0001:C61E       ??_C@_0BA@JEHM@GetOpenFileName?$AA@
 0001:C62E       ??_C@_0BF@GCFH@CommDlgExtendedError?$AA@
 0001:C644       ??_C@_0M@JEJD@LocalServer?$AA@
 0001:C650       ??_C@_0L@KCEB@?$CFc?$CFc?$CFc?4?4?4?2?$AA@
 0001:C65C       ??_C@_04IEDM@LPT1?$AA@
 0001:C662       ??_C@_04HLIF@LPT2?$AA@
 0001:C668       ??_C@_04NBBC@LPT3?$AA@
 0001:C66E       ??_C@_04JCPL@COM1?$AA@
 0001:C674       ??_C@_04GNEC@COM2?$AA@
 0001:C67A       ??_C@_04MHNF@COM3?$AA@
 0001:C680       ??_C@_04JCDA@COM4?$AA@
 0001:C686       ??_C@_03DDP@CON?$AA@
 0001:C68A       ??_C@_03DLI@AUX?$AA@
 0001:C68E       ??_C@_03EHJD@PRN?$AA@
 0001:C692       GETASSOCIATEDEXECUTABLE
 0001:C796       POINTERTONTHFIELD
 0001:C7D4       FICONFILEFROMCLASS
 0001:CAE6       ??_C@_0BE@GGIG@?2Shell?2Open?2Command?$AA@
 0001:CAFA       ??_C@_0BP@CLAL@Protocol?2StdFileEditing?2Server?$AA@
 0001:CB1A       ??_C@_0M@JONA@DefaultIcon?$AA@
 0003:0004       rsrvptrs
 0003:06CC       ?fBeVerbose@@3HE
 0003:0844       _g_dwObjectCount
 0003:0848       _g_dwLockCount
 0003:084C       _uMsgHelp
 0003:084E       _uMsgEndDialog
 0003:0850       _uMsgBrowse
 0003:0852       _uMsgChangeIcon
 0003:0854       _uMsgFileOKString
 0003:0856       _uMsgCloseBusyDlg
 0003:08B4       _STKHQQ
 0003:08B6       __hPrevInstance
 0003:08B8       __hInstance
 0003:08BA       __lpszCmdLine
 0003:08BE       __cmdShow
 0003:08C0       _aseglo
 0003:08C2       _aseghi
 0003:08C4       ___aDBswpflg
 0003:08C6       ___aDBrterr
 0003:08C8       __ctype
 0003:08C8       __ctype_
 0003:09FC       __acfinfo
 0003:0A0A       __aintdiv
 0003:0A0E       __fac
 0003:0A18       _errno
 0003:0A1A       __umaskval
 0003:0A1C       __pspadr
 0003:0A1E       __psp
 0003:0A20       __winminor
 0003:0A20       __winver
 0003:0A21       __winmajor
 0003:0A22       __osver
 0003:0A22       __osminor
 0003:0A23       __osmajor
 0003:0A24       __osversion
 0003:0A26       __osmode
 0003:0A27       __cpumode
 0003:0A28       __doserrno
 0003:0A28       __oserr
 0003:0A2A       __nfile
 0003:0A2C       __wfile
 0003:0A2E       __wnfile
 0003:0A30       __osfile
 0003:0A44       __wsfile
 0003:0A58       ___argc
 0003:0A5A       ___argv
 0003:0A5E       __environ
 0003:0A62       __pgmptr
 0003:0A67       __child
 0003:0A69       __exitflag
 0003:0A6A       __adbgmsg
 0003:0A86       __pnhFarHeap
 0003:0A8A       __qwinused
 0003:0AEE       __fheap
 0003:0AFC       __amblksiz
 0003:0AFE       __aaltstkovr
 0003:0B02       __lastiob
 0003:0B04       __cfltcvt_tab
 0003:0B20       __sigintseg
 0003:0B22       __sigintoff
 0003:0B24       __asizeC
 0003:0B25       __asizeD
 0003:0B26       __cflush
 0003:0B28       __lseekchk
 0003:0B34       __fpinit
 0003:0B44       __iob
 0003:0C34       __iob2
 0003:0ED0       __edata
 0003:0ED0       ?g_cfEmbeddedObject@@3GE
 0003:0ED0       _edata
 0003:0ED2       ?g_cfObjectDescriptor@@3GE
 0003:0ED4       ?lpCSimpleApp@@3PEVCSimpleApp@@E
 0003:1A50       _cfEmbedSource
 0003:1A52       _cfEmbeddedObject
 0003:1A54       _ghInst
 0003:1A56       _cfOwnerLink
 0003:1A58       _cfLinkSrcDescriptor
 0003:1A5A       _cfFileName
 0003:1A5C       _cfLinkSource
 0003:1A5E       _cfObjectDescriptor
 0003:1A60       _end
 0003:1A60       __end

Program entry point at 0001:3384
